:020000040000FA
:100000000C9486190C94AE190C94AE190C94E22D34
:100010000C94AE190C94AE190C94AE190C94AE1944
:100020000C94AE190C94AE190C94AE190C94AE1934
:100030000C94AE190C94AE190C94AE190C94AE1924
:100040000C94982D0C94AE190C94662D0C94402DA4
:100050000C94AE190C94B92E0C94AE190C94AE19E4
:100060000C94AE190C94AE195361766500466C6918
:1000700070004D61696E2053637265656E004F4B71
:10008000004E4F00454E00434E00594553004E4F21
:10009000004F4E004F464600496E666F730042693E
:1000A0006700504944004469726563740053617687
:1000B0006500426F6F7374004F666600536C656530
:1000C00070005361766500426F6F737400536C6506
:1000D00065700044656661756C74005361766500F7
:1000E0004164640044656C6574650052656E616DC1
:1000F000650043616C696272617465004368616E9A
:1001000067650052657475726E0041626F757400A8
:100110004C616E670042757A7A657200536372654E
:10012000656E00436F6E74726F6C0054696D65721A
:100130000054656D70005469700000000000000FED
:100140001DC20800054442080003845FBF000FE49D
:100150004410000115451000054CC97F8009244F4B
:10016000900007C4C11000054D413F000554438174
:100170000007C44D02000544411400055541080024
:1001800007C881040000000000000000000000011A
:10019000083FFE001FFF810000004002000007FE34
:1001A0000FF8000402080800040208880007FE088F
:1001B00088000402088800040208880007FE0888F6
:1001C000000402094800040202300007FE040C008B
:1001D00004021804000000000000000000000001FC
:1001E000100080001FFF80800001103FFF000040D2
:1001F00004080007FC04080004440410000444023E
:10020000100004440220001FFF812000004000C0B5
:100210000000A00130000110020800060C0C0700CD
:100220001803B00200000000000000000000000001
:100230004000800000400080000FFF3FFF000841A9
:1002400004080008410408000841041000084102A5
:1002500010000FFF0220000841012000004000C0F4
:10026000000040013000004002080000400C070080
:100270000040300200000000000000000000001FED
:10028000DF10200002120C20000224042000047F52
:100290008020000424B820000FA488500014BF88D8
:1002A000500004A488500004A488480004BF888833
:1002B0000004A48A880007A48C84000444890700F1
:1002C0000081860200000000000000000000000F16
:1002D000F00491000440025200047F905400045046
:1002E00088FF0007D0848100045100810004490187
:1002F000FF0007CA0281000444048100044A1CFF75
:100300000007EA0481000C510481000061C48500EB
:100310000040808200000000000000000000000794
:10032000FF802000008407FF000084040100008497
:1003300004010000840401000FFFC7FF00008404D3
:1003400000000084040000008405FF000084050113
:100350000001040901000104090100020411FF0069
:100360000404010100000000000000000000000083
:100370008204FF00004402010007FF9021000010EA
:10038000102100001017FD0000101021000FFFD0F9
:100390006100001010A10000281121000028122186
:1003A000000044142100008210A1000301D0450088
:1003B0000C00900200000000000000000000000897
:1003C0004410FE00042810920005FF229200001045
:1003D0003C920000100892001CFE109200041020B5
:1003E000FE0004103E920005FF809200041000926F
:1003F0000005100E92000610309200041000FE005E
:100400000010008200000000000000000000000753
:10041000DF8840000A24104000114210FE00040052
:1004200022820002FF3D020008010A420009F91081
:100430003200090920120009F93E020009090002F0
:100440000009090E020009F9302200080500140015
:100450000802000800000000000000000000000F7B
:10046000C3F1E0000FE3F1F8000C70C19E000C3006
:10047000C186000C30C183000C30C183000C60C108
:1004800083000C60C183000FC0C183000FC0C18610
:10049000000C00C186000C00C198000C03F1F800AC
:1004A0000C03F1E00000000000000000000000006C
:1004B000200820000FFF09FC000020080000002099
:1004C0003E880003FE08500002020BFE0003FE0CF3
:1004D0004000020218400003FE2BFE000202084802
:1004E0000003FE08880002020850000202283000C3
:1004F0001FFF91CC0000000000000104047C0000FC
:10050000880444000FFF3F44000020044400002002
:100510000C440000200E44001FFF954400002014EE
:100520004400005024440000500444000088044566
:10053000000104048500060385030018010400007F
:1005400000000000000000000000000000000004A7
:100550007E21FC0004421104001F7E0904000442B5
:1005600021FC000542110400067E1104000C000568
:10057000FC0015FF880000040813FE0004483252F6
:1005800000044F125200044812520014A8125200E4
:10059000091F97FF0000000000000000000000029B
:1005A000103DFC000210250400041025040005FF86
:1005B000BDFC000C102520000C3825200014382527
:1005C000FE0004543D200004542510000492251020
:1005D000000511A5090006113D4500041025830002
:1005E0000410010100000000000000000000001FD6
:1005F000C8102000124A0C20001AC9042000174815
:100600000020001FFFB8200002080850001FC80883
:100610005000020808500003C80848001E1408884B
:100620000001540A880015220C8400144389070035
:100630000081060200000000000002FE010000022E
:10064000823FFF00048202000004FE0200000C1042
:1006500004FC00141004080005FF8C1000041014A2
:100660001000043825FF0004340410000452041064
:1006700000049184100005100450000410042000B0
:100680000000000000000000000000000000000268
:10069000030010001FDC3EFE00089002120005104F
:1006A00004FF001FDF84120002120CFE001FD202A2
:1006B0001000021222FE000A921410000A521410B6
:1006C0000012220DFF0002220810000A421410003E
:1006D000040223FF00000000000000000000000FE3
:1006E00078BC20000948A45000094AA85000094AD3
:1006F000A88800094AB104001FFEAAFB00094AA409
:100700002000094AA42000094AA7FE00094AB42093
:10071000000948A924000B48A22200088AA4A200CC
:10072000111920400000000000000000000000003F
:1007300020008000005001FC00008801040001043A
:1007400003080006FB0490000800C0600007DF01FA
:100750008000045106000004511BFE0004510202F7
:100760000007D90202000456020200001003FE0036
:100770000010020200000000000000000000000263
:1007800008209000027F9890001F8009FF0002223D
:1007900001100006218B100007628DFE000AA209DD
:1007A00010000A14111000121431FE00020811107A
:1007B0000002141110000222111000024391FF00E8
:1007C0000281110000000000000000000000001085
:1007D0000700000008F83FFE0004802002000080AF
:1007E00020020000BE23E2001C8222220004A42278
:1007F000220004942222000488222200049423E28E
:1008000000052220020005422002000A003FFE00EF
:1008100011FFA00200000000000000000000000125
:10082000041FFC0000880080000FFF0080000020F3
:10083000008000002000800000203FFF001FFF809C
:1008400080000020008000005000800000500080E8
:100850000000880080000104008000060382800000
:100860001801010000000000000009FF0040000422
:10087000203FFF00042000000000FE0000001C429A
:100880000FFC00044200000007FF80000004000F7E
:10089000FC0004FF000000048100000005810FFC43
:1008A00000068108040004FF08040000810FFC001A
:1008B0000000000000000000000000000000000038
:1008C000400080001FFF9FFC0000400410000FFF4D
:1008D00002200000003FFF000FFE00000008420F52
:1008E000F80008420808000FFE08080008020FF888
:1008F000000800080800080008080008000FF800B9
:1009000010000808000000000000000000000007C0
:10091000FE0FF8000402000000040200000007FEC1
:1009200000000004023FFE00040200800007FE00F9
:100930008000009004900008910C880006931086B7
:10094000000294208200009000800000900280004D
:100950001FFF8100000000000000000000000004F4
:100960001012020005FF9FD20005009212001E28FF
:10097000A2120004443FF2000482021200060002A8
:1009800012000CFE1FD2001410125200041012426A
:10099000000410134200041012820015FF820A00A6
:1009A0000800020400000000000000000000000039
:1009B0002000000000203E04001FFFA204001000E1
:1009C000A2FF0000012204000FFE22040000403EAE
:1009D000440000402224000440222400047C22041D
:1009E0000004402204000A403E0400094022240082
:1009F00010FF80140000000008000000000000103C
:100A0000FE08200008820BFF0004820A010010FE8D
:100A10003C51000882088800088209040002FE0C8C
:100A20000000040019FC0009FF28200019290820F3
:100A3000000929082000092908200009292BFF00A6
:100A40000BFF900000000000000000000000001FED
:100A50007F90F80001080888000A10088800047FC9
:100A60000107001FC13A0000054909FC00044908BC
:100A700084000449088800044908480004490850D3
:100A80000004490A200004160C580014218987002C
:100A900008C086020000000000000FFFFFFFFFF00B
:100AA0003FFFFFFFFFFC7FFFFFFFFFFE7FFFFFFF1A
:100AB000FFFEF0000000000FF0000000000FF0004B
:100AC0000000000FF1FFFFFFFF8FF1FFFFFFFF8F1F
:100AD000F1FFFFFFFF8FF1FFFFFFFF8FF1FFFFFF30
:100AE000FF8FF1FFFFFFFF8FF1FFFFFFFF8FF1FF90
:100AF000FFFFFF8FF1FFFFFFFF8FF1FFFFFFFF8F72
:100B0000F1FFFFFFFF8FF1FFFFFFFF8FF1FFFF03FB
:100B1000FF8FF1FFFF03FF8FF1FFFF03FF8FF1FF57
:100B2000FFFFF18FF1FFFFFFE18FF1FFFFFFC78FA5
:100B3000F1FFFFFF8F8FF1FFFFFF0F8FF1FFFFFF2F
:100B40008F8FF1FFFFFFC78FF1FFFFFFE18FF1FFF5
:100B5000FFFFF18FF1FFFFFFFF8FF1FFFFFFFF8F1F
:100B6000F0000000000FF0000000000FF000000097
:100B7000000FF1FFFFFFFF8FF1111FFFFF8FF1113A
:100B80001FFFFF8FF1111FFFFF8FF1FFFFFFFF8F8F
:100B9000F0000000000FF0000000000FF000000067
:100BA000000F7FFFFFFFFFFE7FFFFFFFFFFE3FFF06
:100BB000FFFFFFFC0FFFFFFFFFF00FFFFFFFFFF046
:100BC0003FFFFFFFFFFC7FFFFFFFFFFE7FFFFFFFF9
:100BD000FFFEFFFFFFFFFFFFFFFFFFFFFFFFFFFF26
:100BE000FFFFFFFFFFFFFFFFFFFFFFFFFFFFFFFF15
:100BF000FFFFFFFFFFFFFFFFFFFFFFFFFFFFFFFF05
:100C0000FFFFFFFFFFFFFFFFFFFFFFFFFFFFFFFFF4
:100C1000FFC7001FC00FFFC7001FC00C1FC7001F6A
:100C2000C00C1FC71FFFC7FC0FC71FFFC7FC4FC764
:100C30001FFFC7FC4FC71FFFC7FC47C71FFFC7FCED
:100C400067C71C01C01C63C71C01C01C73C71C0103
:100C5000C01C71C71F8FC7FC79C71F8FC7FC78C71F
:100C60001F8FC7FC7C071F8FC7FC7C07000FC00CC1
:100C70007E07000FC00FFFFF000FC00FFFFFFFFF39
:100C8000FFFFFFFFFFFFFFFFFFFFFFFFFFFFFFFF74
:100C9000FFFFFFFFFFFFFFFFFFFFFFFFFFFFFFFF64
:100CA000FFFFFFFFFFFFFFFFFFFFFFFFFFFFFFFF54
:100CB000FFFFFFFFFFFFFFFFFFFFFFFFFFFFFFFF44
:100CC000FFFF7FFFFFFFFFFE7FFFFFFFFFFE3FFFF6
:100CD000FFFFFFFC0FFFFFFFFFF00FFFFFFFFFF025
:100CE0003FFFFFFFFFFC7FFFFFFFFFFE7FFFFFFFD8
:100CF000FFFEFFFFFFFFFFFFFFFFFFFFFFFFFFFF05
:100D0000FFFFFFFFFFFFFC7FFFFFFFFFFC7FFFFFF9
:100D1000FFFFFC7FFFFFFFFFFC7FFFFFFFFFFC7F6C
:100D2000FFFFFFFFFC7FFFFFFFFFFC7FFFFFFFFFD9
:100D3000FC7FFFFFFE00000001FFFE00000001FF3E
:100D4000FE00000001FFFE3FFC7FF1FFFE3FFC7F45
:100D5000F1FFFE3FFC7FF1FFFE3FFC7FF1FFFE3F16
:100D6000FC7FF1FFFE3FFC7FF1FFFE3FFC7FF1FFC8
:100D7000FE3FFC7FF1FFFE3FFC7FF1FFFE00000025
:100D8000007FFE000000007FFE000000007FFE3FAD
:100D9000FC7FFFFFFFFFFC7FFFFFFFFFFC7FFFFFEC
:100DA000FFFFFC7FFFFFFFFFFC7FFFFFFFFFFC7FDC
:100DB000FFFFFFFFFC7FFFFFFFFFFC7FFFFFFFFF49
:100DC000FC7FFFFFFFFFFC7FFFFFFFFFFC7FFFFFBC
:100DD000FFFFFCFFFFFFFFFFFFFFFFFFFFFFFFFF26
:100DE000FFFF7FFFFFFFFFFE7FFFFFFFFFFE3FFFD5
:100DF000FFFFFFFC0FFFFFFFFFF00FFFFFFFFFF004
:100E00003FFFFFFFFFFC7FFFFFFFFFFE7FFFC003F1
:100E1000FFFEFFFF0000FFFFFFFC00003FFFFFF0B1
:100E200000000FFFFFC0000003FFFFC0000001FF34
:100E3000FF00000000FFFF000000007FFE00000038
:100E4000007FFC000000003FFC000000203FF80095
:100E50000000701FF8000000F81FF0000001F80FFC
:100E6000F0000003F00FF0000007E00FF000000FAB
:100E7000C00FE000001F8007E001803F0007E00393
:100E8000C07E0007E007E0FC0007E003F1F8000780
:100E9000E001FFF00007E000FFE00007E0007FC096
:100EA0000007F0003F80000FF0001F00000FF0006F
:100EB0000E00000FF0000400000FF8000000001FFB
:100EC000F8000000001FFC000000003FFC000000D4
:100ED000003FFF000000007FFF00000000FFFF80D8
:100EE000000001FFFFC0000003FFFFF0000007FF4C
:100EF000FFF000000FFFFFFC00003FFFFFFF0000BE
:100F0000FFFF7FFFF00FFFFE7FFFFFFFFFFE3FFFB2
:100F1000FFFFFFFC0FFFFFFFFFF00FFFFFFFFFF0E2
:100F20003FFFFFFFFFFC7FFFFFFFFFFE7FFFC001D2
:100F3000FFFEFFFF0000FFFFFFFC00001FFFFFF0B0
:100F400000000FFFFFE0000003FFFFC0000001FFF3
:100F5000FF80000000FFFF000000007FFE00000097
:100F6000007FFE000000003FFC008000801FF801B1
:100F7000C003C01FF803E003E01FF803F00FE00F09
:100F8000F001F80FC007F000FC1F8007F0007E7F23
:100F90000007E0003FFE0007E0001FFC0007E00044
:100FA0000FF80007E00007F00007E00007F0000777
:100FB000E0001FF80007E0001FFC0007E0007FFED4
:100FC0000007F0007E3F0007F001FC1F8007F001E2
:100FD000F80FC00FF803F007E00FF803E003E01F7D
:100FE000F801C001801FFE008000803FFE0000006D
:100FF000003FFF000000007FFF000000007FFF8037
:10100000000000FFFFC0000001FFFFF0000007FF2D
:10101000FFF800000FFFFFFC00003FFFFFFF800014
:10102000FFFF7FFFF007FFFE7FFFFFFFFFFE3FFF99
:10103000FFFFFFFC0FFFFFFFFFF00FFFFFFFFFF0C1
:101040003FFFFFFFFFFC7FFFFFFFFFFE7FFFF00F73
:10105000FFFEFFFFF00FFFFFFFFFE007FFBFFFFFF7
:10106000C3C3FF1FFFFF87E1FE0FFFFF0FF0FC1F51
:10107000FFFE1FF8783FFFFC3FFCF07FFFF87FFF8B
:10108000E0FFFFF0FFFFC1FFFFE1FFFF83FFFFE392
:10109000FFFF07FFFFE3FFFE07FFFFE3FFFC07FF84
:1010A000FFE3FFF807FFFFE3FFF047FFFFE3FFE089
:1010B000C7FFFFE3FFC1C7FFFFE3FF83C7FFFFE3F6
:1010C000FF07C7FFFFE3FE0FC7FFFFE3FC1FC7FFDC
:1010D000FFE3F83FC7FFFFE3F07FC7FFFFE3E0FF59
:1010E000C7FFFFE3C1FFC7FFFFE783FFC7FFFFEFB6
:1010F00007FFC7FFFFFE0FFFC1FFFFFC1FFFE0FF61
:10110000FFF83FFFF87FFFF07FFFFC3FFFE00000AC
:10111000003FFFC00000003FFF800000003FFF07CE
:10112000FFFFFFFFFE0FC003FFFFFC1FC003FFFF19
:10113000FE3FE007FFFFFF7FE007FFFFFFFFF81F15
:10114000FFFF7FFFF81FFFFE7FFFFFFFFFFE3FFF58
:10115000FFFFFFFC0FFFFFFFFFF00FFFFFFFFFF0A0
:101160003FFFFFFFFFFC7FFFFFFFFFFE7FFFFFFF53
:10117000FFFEF0000000000FF0000000000FF00084
:101180000000000FF1FFFFFFFF8FF1FFFFF8888FD6
:10119000F1FFFFF8888FF1FFFFF8888FF1FFFFFF65
:1011A000FF8FF0000000000FF0000000000FF000C3
:1011B0000000000FF1FFFFFFFF8FF10DDDFE4A8FF2
:1011C000F10AAAFFCD8FF10888FE5F8FF11AAAFFFE
:1011D000FF8FF1FFFFFFFF8FF1FFFFFFFF8FF1FF99
:1011E000FF00008FF10C017FFF8FF16FFF46318F01
:1011F000F16C3F56B78FF11FFF56B78FF1FFFF46D7
:10120000318FF1FFFF77B58FF1FFFF77B58FF10CCD
:101210000177B58FF16FFF46318FF16C3F7FFF8F04
:10122000F11FFF00008FF1FFFFFFFF8FF1FFFFFFB6
:10123000FF8FF1FFFFFFFF8FF100002AA48FF10065
:101240000055228FF1E0002AA48FF1FFFFFFFF8FEE
:10125000F0000000000FF0000000000FF0000000A0
:10126000000F7FFFFFFFFFFE7FFFFFFFFFFE3FFF3F
:10127000FFFFFFFC0FFFFFFFFFF00FFFFFFFFFF07F
:101280003FFFFFFFFFFC7FFFFFFFFFFE7FFFFFFF32
:10129000FFFEF0000000000FF0000000000FF00063
:1012A0000000000FF1FFFFFFFF8FF1FFFFF8888FB5
:1012B000F1FFFFF8888FF1FFFFF8888FF1FFFFFF44
:1012C000FF8FF0000000000FF0000000000FF000A2
:1012D0000000000FF1FFFFFFFF8FF1FFFFFFFF8F07
:1012E000F1FFFFFFFF8FF1FFFFFFFF8FF1FFFFFF18
:1012F000FF8FF180F01F018FF180F01F018FF19CB3
:10130000F39FF98FF19CF39FF98FF19CF39FF98F75
:10131000F19CF39FF98FF180F01C018FF180F01C9C
:10132000018FF1FCFF9CF98FF1FCFF9CF98FF1FC20
:10133000FF9CF98FF1FCFF9CF98FF100E01C018FFD
:10134000F100E01C018FF1FFFFFFFF8FF1FFFFFFB6
:10135000FF8FF1FFFFFFFF8FF1FFFFFFFF8FF1FF17
:10136000FFFFFF8FF1FFFFFFFF8FF1FFFFFFFF8FF9
:10137000F0000000000FF0000000000FF00000007F
:10138000000F7FFFFFFFFFFE7FFFFFFFFFFE3FFF1E
:10139000FFFFFFFC0FFFFFFFFFF00FFFFFFFFFF05E
:1013A0003FFFFFFFFFFC7FFFFFFFFFFE7FFFFFFF11
:1013B000FFFEFFFFFFFFFFFFFDFFFFFFFFFFF8FF47
:1013C000FFFFFFFFF07FFFFFFFFFE03FFFFFFFFF9B
:1013D000F8FFFFFFFFFFF8FFFFFFFFFFF8FFFFFF32
:1013E000FFFFF8E7FFFFFFFFF8E7FFE1FFFFF8E38C
:1013F000FF007FFFF8F3FE0C1FFFF8F3F87F0FFFED
:10140000F8F1F0FFC7FFF8F9E3FFE3FFF8F8E7FFB3
:10141000F1FFF8FC47FFF8FFF8FE0FFFFCFFF8FFB5
:101420001FFFFFFFF8FF1FFFFFFFF8FE0FFFFFFF8B
:10143000F8FE47FFFFFFF8FC63FFFFFFF8FCF0FF3B
:10144000FFFFF8F8F87FFFFFF8F9FE1FFFFFF8F144
:10145000FF07FFFFF8E3FFC1FFFFF8C7FFF01FFF23
:10146000F8C7FFFC07FFF8CFFFFFC7FFF8FFFFFF3C
:10147000FFFFF8FFFFFFFFFFF8FFFFFFFFBFF8FFD1
:10148000FFFFFF9FF8000000000FF80000000007BA
:10149000F8000000000FFFFFFFFFFF9FFFFFFFFFAF
:1014A000FFBF7FFFFFFFFFFE7FFFFFFFFFFE3FFF4E
:1014B000FFFFFFFC0FFFFFFFFFF00FFFFFFFFFF03D
:1014C0003FFFFFFFFFFC7FFFFFFFFFFE7FFFFFFFF0
:1014D000FFFEFFFFFFFFFFFFFDFFFFFFFFFFF8FF26
:1014E000FFFFFFFFF07FFFFFFFFFE03FFFFFFFFF7A
:1014F000F8FFFFFFFFFFF8FFFFFFFFFFF8FFFFFF11
:10150000FFFFF8E7FFFFFFFFF8E7C00003FFF8E386
:10151000C00003FFF8F3CFFFFFFFF8F3CFFFFFFF9B
:10152000F8F1CFFFFFFFF8F9CFFFFFFFF8F8CFFF8B
:10153000FFFFF8FC4FFFFFFFF8FE0FFFFFFFF8FF74
:101540000FFFFFFFF8FF0FFFFFFFF8FF8FFFFFFF09
:10155000F8FFC7FFFFFFF8FFC3FFFFFFF8FFC0FF63
:10156000FFFFF8FFC87FFFFFF8800E1FFFFFF88026
:101570000F07FFFFF8FFFFC1FFFFF8FFFFF01FFF9E
:10158000F8FFFFFC07FFF8FFFFFFC7FFF8FFFFFFB3
:10159000FFFFF8FFFFFFFFFFF8FFFFFFFFBFF8FFB0
:1015A000FFFFFF9FF8000000000FF8000000000799
:1015B000F8000000000FFFFFFFFFFF9FFFFFFFFF8E
:1015C000FFBF7FFFFFFFFFFE7FFFFFFFFFFE3FFF2D
:1015D000FFFFFFFC0FFFFFFFFFF00FFFFFFFFFF01C
:1015E0003FFFFFFFFFFC7FFFFFFFFFFE7FFFFE3F90
:1015F000FFFEFFFFFE3FFFFFFFFFFE3FFFFFFFFF7E
:10160000FE3FFFFFFFFFFE3FFFFFFFFFBE3DFFFF6F
:10161000FFFE3E3C7FFFFFFC3E3C3FFFFFF83E3CB1
:101620001FFFFFF0FE3F0FFFFFE1FE3F87FFFFC3FD
:10163000FE3FC3FFFF87FE3FE1FFFF8FFE3FF1FF4D
:10164000FF0FFE3FF0FFFF1FFE3FF8FFFF1FFE3FB3
:10165000F8FFFE1FFE3FFC7FFE3FFE3FFC7FFE3F8C
:10166000FE3FFC7FFE3FFE3FFC7FFE3FFE3FFC7FD8
:10167000FE3FFFFFFC7FFE3FFFFFFC7FFE1FFFFFE3
:10168000FC7FFF1FFFFFF8FFFF1FFFFFF8FFFF0FAB
:10169000FFFFF0FFFF8FFFFFF1FFFF87FFFFE1FF7D
:1016A000FFC3FFFFC3FFFFE1FFFF87FFFFF0FFFF67
:1016B00007FFFFF83FFC0FFFFFFC0FF03FFFFFFEAF
:1016C00000007FFFFFFF8001FFFFFFFFF00FFFFF24
:1016D000FFFFFFFFFFFFFFFFFFFFFFFFFFFFFFFF1A
:1016E000FFFF7FFFFFFFFFFE7FFFFFFFFFFE3FFFCC
:1016F000FFFFFFFC0FFFFFFFFFF00FFFFFFFFFF0FB
:101700003FFFFFFFFFFC7FFEFFFFFFFE7FFE7FFF2F
:10171000FFFEFFFE3FFFFFFFFFFE1FFFFFFFFFFE7D
:101720000FFFFFFFFFFE07FFFFFFFFFE03FFFFFFAF
:10173000FFFE01FFFFFFFFFE01FFFFFFFFFC00FFB9
:10174000FFFFFFF800FFFFFFFFF000FFFFFFFFE0DC
:10175000007FFFFFFFE0007FFFFFFFC0007FFFFF74
:10176000FF80007FFFFFFF00007EFFFFFF00007E85
:101770007FFFFE0000FE3FFFFC0000FF1FFFFC009C
:1017800000FE0FFFF80001FE07FFF80001FE03FF57
:10179000F00003FC01FFF00007FC01FFF0000FF870
:1017A00001FFF0001FF000FFF0001FF000FFF0004D
:1017B0003FE0007FF8007FC0007FF800FF80007FDF
:1017C000FC00FF00007FFC01FF00007FFE01FE0027
:1017D000007FFE03FC00007FFF03F80000FFFF8393
:1017E000F80000FFFFC7F80000FFFFE3F00001FF73
:1017F000FFF3F00003FFFFFFF00007FFFFFFFFFF15
:10180000FFFF7FFFFFFFFFFE7FFFFFFFFFFE3FFFAA
:10181000FFFFFFFC0FFFFFFFFFF00FFFFFFFFFF0D9
:101820003FFFFFFFFFFC7FFFFFFFFFFE7FFFFFC1CA
:10183000FFFEFFFFFF01FFFFFFFFFC01FFFFFFFFB8
:10184000F001FFFFFFFFC001FFFFFFFF0007FFFFE9
:10185000FFFC001FFFFFFFF0007F9FFFFFE001FE86
:101860000FFFFFC007F807FFFFC01FE007FFFFC023
:101870007F8007FFFFE1FE001FFFFFFFF8003FFF33
:10188000FFFFE001FFFFFFFF8003FFFFFFFE000FF0
:10189000FFFFFFF8003FFFFFFFE000FE0FFFFFC06C
:1018A00003FC07FFFFC00FE007FFFFC03FC007FFBB
:1018B000FFC0FE000FFFFFFFFC003FFFFFFFE00047
:1018C0007FFFFFFFC003FFFFFFFF0001FFFFFFFEE1
:1018D0000001FFFFFFFE0000FFFFFFFE0001FFFF12
:1018E000FFFF0001FFFFFFFFFFFFFFFFFFFFFFFF05
:1018F000FFFFFFFFFFFFFFFFFFFFFFFFFFFFFFFFF8
:10190000FFFFFFFFFFFFE00FFFFFFFFFC007FFFF2D
:10191000FFFF8007FFFFFFFF8007FFFFFFFFC00FF4
:10192000FFFF7FFFE01FFFFE7FFFFFFFFFFE3FFF88
:10193000FFFFFFFC0FFFFFFFFFF00FFFFFFFFFF0B8
:101940003FFFFFFFFFFC7FFFFFFFFFFE7FFFFFFF6B
:10195000FFFEF00000001FFFF00000000FFFF0008E
:10196000000007FFF1C00FF8C3FFF1C00FF8E1FF5F
:10197000F1C00FF8F0FFF1C00FF8F87FF1C00FF8D9
:10198000FC3FF1C00FF8FE1FF1C00000FF0FF1C0D7
:101990000000FF8FF1C00000FF8FF1FFFFFFFF8FFE
:1019A000F1FFFFFFFF8FF1FFFFFFFF8FF1FFFFFF51
:1019B000FF8FF1FFFFFFFF8FF1FFFFFFFF8FF1FFB1
:1019C000FFFFFF8FF1FFFFFFFF8FF1FFFFFFFF8F93
:1019D000F1C00000038FF1C00000038FF1C00000D0
:1019E000038FF1C7FFFFE38FF1C7FFFFE38FF1C65E
:1019F0000000E38FF1C60000E38FF1C60000E38F23
:101A0000F1C7FFFFE38FF1C7FFFFE38FF1C60000CF
:101A1000E38FF1C60000E38FF1C60000E38FF1C74A
:101A2000FFFFE38FF1C7FFFFE38FF1C7FFFFE38FF6
:101A3000F0000000000FF0000000000FF0000000B8
:101A4000000F7FFFFFFFFFFE7FFFFFFFFFFE3FFF57
:101A5000FFFFFFFC0FFFFFFFFFF00FFFFFFFFFF097
:101A60003FFFFFFFFFFC7FFFFFFFFFFE7FFFFFFF4A
:101A7000FFFEFFFFFFFFFFFFFFFFFFFFFFFFFFFF77
:101A8000FFFFFFFFFFFFFFFFFFFFFFFFFFFFFFFF66
:101A9000FFFFFFFFFFFFFFFFFFFFFFFFFFFFFE3F17
:101AA000FFFFFFFFFE3FFFFFFFFFFE3FFFFFFFFFC8
:101AB000FE3FFFFFFFFFFE3FFFFFFFFFFE3FFFFF79
:101AC000FFFFFE3FFFFFFFFFFE3FFFFFFFFFFE3F69
:101AD000FFFFFFFFFE3FFFFFFFFFFE3FFFFFFFF0A7
:101AE00000000FFFFFF000000FFFFFF000000FFFEE
:101AF000FFFFFFFFFFFFFFFFFE3FFFFFFFFFFE3F78
:101B0000FFFFFFFFFE3FFFFFFFFFFE3FFFFFFFFF67
:101B1000FE3FFFFFFFFFFE3FFFFFFFFFFE3FFFFF18
:101B2000FFFFFE3FFFFFFFFFFE3FFFFFFFFFFFFF47
:101B3000FFFFFFFFFFFFFFFFFFFFFFFFFFFFFFFFB5
:101B4000FFFFFFFFFFFFFFFFFFFFFFFFFFFFFFFFA5
:101B5000FFFFFFFFFFFFFFFFFFFFFFFFFFFFFFFF95
:101B6000FFFF7FFFFFFFFFFE7FFFFFFFFFFE3FFF47
:101B7000FFFFFFFC0FFFFFFFFFF00FFFFFFFFFF076
:101B80003FFE00007FFC7FFE00007FFE7FFC000028
:101B90003FFEFFFC7FFE3FFFFFFC7FFE3FFFFFFCA1
:101BA0007FFE3FFFFC000000001FF8000000000F58
:101BB000F00000000007F1FFFFFFFFC7F1FFFFFF8C
:101BC000FFC7F1FFFFFFFFC7F00000000007F800AC
:101BD0000000000FFC000000001FFFFFFFFFFFFFE1
:101BE000FC7FFFFFFE3FFC7FFFFFFE3FFC7FFFFF10
:101BF000FE3FFC7F8FF8FE3FFC7F8FF8FE3FFC7FAF
:101C00008FF8FE3FFC7F8FF8FE3FFC7F8FF8FE3F92
:101C1000FC7F8FF8FE3FFC7F8FF8FE3FFC7F8FF844
:101C2000FE3FFC7F8FF8FE3FFC7F8FF8FE3FFC7F7E
:101C30008FF8FE3FFC7F8FF8FE3FFC7F8FF8FE3F62
:101C4000FC7F8FF8FE3FFC7F8FF8FE3FFC7F8FF814
:101C5000FE3FFC7F8FF8FE3FFC7FFFFFFE3FFC7FD7
:101C6000FFFFFE3FFC7FFFFFFE3FFC7FFFFFFE3FCD
:101C7000FC7FFFFFFE3FFC3FFFFFFC3FFC0000003E
:101C8000003F7E000000007E7F00000000FE3FFF5E
:101C9000FFFFFFFC0FFFFFFFFFF00FFFFFFFFFF055
:101CA0003FFFFFFFFFFC7FFFFFFFFFFE7FFFFFFF08
:101CB000FFFEFFFFFFFFFFFFFFFFFFFFFFFFFFFF35
:101CC000FFFFFFFFFFFFF007FFFFFFFF8000FFFFA9
:101CD000FFFE00003FFFFFF807F00FFFFFF03FFEA1
:101CE00007FFFFE0FFFF83FFFFC1FFFFE1FFFF876B
:101CF000FFFFF0FFFF0FFFFFF87FFF0FFFFFFC7FED
:101D0000FE1FFFFFFC3FFE3FFFFFFE3FFC3FF3FBDC
:101D1000FE1FFC7FE1F0FF1FFC7FC0E07F1FF87F0C
:101D200080407F0FF8FF00003F8FF8FF00003F8FDB
:101D3000F8FF00001F8FF8FE00001F8FFFFE00005D
:101D40001FFFFFFE00001FFFFFFE00001FFFFFFF41
:101D500000001FFFFFFF00003FFFFFFF00003FFFED
:101D6000FFFF80007FFFFFFF80007FFFFFFFC000BD
:101D7000FFFFFFFFF003FFFFFFFFFC0FFFFFFFFF71
:101D8000FFFFFFFFFFFFFFFFFFFFFFFFFFFFFFFF63
:101D9000FFFFFFFFFFFFFFFFFFFFFFFFFFFFFFFF53
:101DA000FFFF7FFFFFFFFFFE7FFFFFFFFFFE3FFF05
:101DB000FFFFFFFC0FFFFFFFFFF00FFFFFFFFFF034
:101DC0003FFFFFFFFFFC7FFFFFFFFFFE6000000003
:101DD0001FFEE00000001FFFE00000001FFFE3FF08
:101DE000FFFF1FFFE3FFFFFF1FFFE3FFFFFF10FFEA
:101DF000E3FFFFFF10FFE3FFFFFF10FFE3FFFFFF25
:101E000018FFE3FFFFFF18FFE3FFFFFF1887E3FF63
:101E1000FFFF1887E3FFFFFF1887E3FFFFFF18C7E7
:101E2000E3FFFFFF18C7E3FFFFFF18C7E3FFFFFF54
:101E300018C7E3FFFFFF18C7E3FFFFFF18C7E3FF63
:101E4000FFFF18C7E3FFFFFF18C7E3FFFFFF18C737
:101E5000E3FFFFFF18C7E3FFFFFF18C7E3FFFFFF24
:101E600018C7E3FFFFFF18C7E3FFFFFF18C7E3FF33
:101E7000FFFF18C7E3FFFFFF18C7E000000018C707
:101E8000E000000018C7E000000018C7FFFFFFFFD8
:101E9000F8C7FF1FFFFFF8C7FF00000000C7FF00E3
:101EA000000000C7FF00000000C7FFFFFFFFFFC7E3
:101EB000FFF8FFFFFFC7FFF800000007FFF8000072
:101EC00000077FF8000000067FFFFFFFFFFE3FFFD7
:101ED000FFFFFFFC0FFFFFFFFFF00FFFFFFFFFF013
:101EE0003FFFFFFFFFFC7FFFFFFFFFFE7FFFFFFFC6
:101EF000FFFEFFFFFFFFFFFFF000007FFFFFF0008E
:101F0000007FFFFFF000007FFFFFF1FFFFFFFF0FEB
:101F1000F1FFFFFFFE0FF1FFFFFFFC0FF1FFFFFFDF
:101F2000F81FF1FFFFFFF03FF1FFFFFFE07FF1FF40
:101F3000FFFFC0FFF1FFFFFF81FFF1FFFFFF03FF86
:101F4000F1FFFFFE07FFF1FFFFFC0FFFF1FE1FF89F
:101F50001FFFF1FE0FF03FFFF1FE07E07FFFF1FEF4
:101F600003C0FFFFF1FF0181FFFFF1FF8003FFFFCF
:101F7000F1FFC007FC7FF1FFE00FFC7FF1FFF01FD6
:101F8000FC7FF1FFF83FFC7FF1FFFC7FFC7FF1FF5E
:101F9000FFFFFC7FF1FFFFFFFC7FF1FFFFFFFC7FF6
:101FA000F1FFFFFFFC7FF1FFFFFFFC7FF1FFFFFF71
:101FB000FC7FF1FFFFFFFC7FF1FFFFFFFC7FF1FFE4
:101FC000FFFFFC7FF0000000007FF0000000007FBA
:101FD000F0000000007FFFFFFFFFFFFFFFFFFFFF9C
:101FE000FFFF7FFFFFFFFFFE7FFFFFFFFFFE3FFFC3
:101FF000FFFFFFFC0FFFFFFFFFF00FFFFFFFFFF0F2
:102000003FFFFFFFFFFC7FFFFFFFFFFE7FFFFFFFA4
:10201000FFFEFFFFFFFFFFFFFFFFFF1FFFFFFFFFB1
:10202000FE0FFFFFFFFFFE0FFFFFFFFFFE0FFFFF93
:10203000FFFFFF1FFFFFFFFFFFFFFFFFFFFFFFFF90
:10204000FFFFFFFFFFFFFFFFFFFFFFFFFFFFFFFFA0
:10205000FFFFFFFFFFFFC00FFFFFFFFF8007FFFF36
:10206000FFFF0007FFFFFFFE0F87FFFFFFFE1FC7F9
:10207000FFFFFFFE3FC7FFFFFFFE3FC7FFFFFFFF62
:10208000FFC7FFFFFFFFFFC7FFFFFFFFFFC7FFFF08
:10209000FFFFFF87FFFFFFFFFF0FFFFFFFFFFE1F99
:1020A000FFFFFFFFFC3FFFFFFFFFF87FFFFFFFFF8A
:1020B000F0FFFFFFFFFFF1FFFFFFFFFFF1FFFFFF5B
:1020C000FFFFF1FFFFFFFFFFF1FFFFFFFFFFF1FF4A
:1020D000FFFFFFFFF1FE3FFFFFFFF0FE3FFFFFFFAF
:1020E000F87C3FFFFFFFFC003FFFFFFFFE007FFF8C
:1020F000FFFFFF00FFFFFFFFFFFFFFFFFFFFFFFFEF
:10210000FFFF7FFFFFFFFFFE7FFFFFFFFFFE3FFFA1
:10211000FFFFFFFC0FFFFFFFFFF00FFFFFFFFFF0D0
:102120003FFFFFFFFFFC7FFFC001FFFE7FFE0000BF
:102130007FFEFFF800001FFFFFE0000007FFFFC069
:10214000400203FFFF81800181FFFF078420E0FF41
:10215000FE0F0C30F07FFC1E0C38783FF83E1C3828
:102160007C1FF87C1C3C3E1FF07C3C3C3F0FF0FC8D
:102170003C3E1F0FE1F87C3E1F87E1F87C3E1F8745
:10218000E1F87C3F1FC7C3F8FC3F0FC3C3F0FC3F1F
:102190000FC3C3F0FC3F0FC3C00000000003C0002A
:1021A00000000003C00000000003C00000000003A6
:1021B000C7F0FC3F0FE3C3F0FC3F0FE3C3F0FC3F6D
:1021C0000FC3C3F0FC3F0FC3C3F0FC3F0FC3E1F8E4
:1021D000FC3F1FC7E1F87C3E1F87E1F87C3E1F876C
:1021E000F0FC7C3E3F0FF07C3C3C3E0FF87C3C3CDE
:1021F0003E1FFC3E1C387C3FFC1E0C30783FFE0F1F
:102200000C30F07FFF030420C0FFFF81800181FFBD
:10221000FFC0000003FFFFF000000FFFFFF8000009
:102220001FFF7FFE00007FFE7FFFC003FFFE3FFF1A
:10223000FFFFFFFC0FFFFFFFFFF00FFFFFFFFFF0AF
:102240003FFFFFFFFFFC7FFFFFFFFFFE7FFFF00F61
:10225000FFFEFFFFF00FFFFFFFFFE007FFFFFFFFA5
:10226000C3C3FFFFFFFF87E1FFFFFFFF0FF0FFFF8B
:10227000FFFE1FF87FFFFFFC3FFC3FFFFFF87FFEE4
:102280001FFFFFF0FFFF0FFFFFE1FFFF87FFFFE3EF
:10229000FFFFC7FFFFE3FFFFC7FFFFE3FFFFC7FF2E
:1022A000FFE3FFFFC7FFFFE3FFFFC7FFFFE3FFFF02
:1022B000C7FFFFE3FFFFC7FFFFE3FFFFC7FFFFE32A
:1022C000FFFFC7FFFFE3FFFFC7FFFFE3FFFFC7FFFE
:1022D000FFE3FFFFC7FFFFE3FFFFC7FFFFE3FFFFD2
:1022E000C7FFFFE3FFFFC7FFFFE3FFFFC7FFFFE3FA
:1022F000FFFFC7FFFF83FFFFC1FFFF07FFFFE0FFF7
:10230000FE1FFFFFF87FFC3FFFFFFC3FFC000000CB
:10231000003FFC000000003FFC000000003FFFFF0A
:10232000FFFFFFFFFFFFC003FFFFFFFFC003FFFF33
:10233000FFFFE007FFFFFFFFE007FFFFFFFFF81FC2
:10234000FFFF7FFFF81FFFFE7FFFFFFFFFFE3FFF46
:10235000FFFFFFFC0FFFFFFFFFF00FFFFFFFFFF08E
:102360003FFFFFFFFFFC7FFFFFFFFFFE7FFFFFFF41
:10237000FFFEF0000000000FF0000000000FF00072
:102380000000000FF1FFFFFFFF8FF1FFFFF8888FC4
:10239000F1FFFFF8888FF1FFFFF8888FF1FFFFFF53
:1023A000FF8FF0000000000FF0000000000FF000B1
:1023B0000000000FF1FFFFFFFF8FF1FFFFFFFF8F16
:1023C000F18FFFFFFF8FF187FFFFFF8FF1E3FFFF2B
:1023D000FF8FF1F1FFFFFF8FF1F0FFFFFF8FF1F1B2
:1023E000FFFFFF8FF1E3FFFFFF8FF187FFFFFF8FFD
:1023F000F18FFFFFFF8FF1FFC0FFFF8FF1FFC0FFE5
:10240000FF8FF1FFC0FFFF8FF1FFFFFFFF8FF1FF95
:10241000FFFFFF8FF1FFFFFFFF8FF1FFFFFFFF8F38
:10242000F1FFFFFFFF8FF1FFFFFFFF8FF1FFFFFFC6
:10243000FF8FF1FFFFFFFF8FF1FFFFFFFF8FF1FF26
:10244000FFFFFF8FF1FFFFFFFF8FF1FFFFFFFF8F08
:10245000F0000000000FF0000000000FF00000008E
:10246000000F7FFFFFFFFFFE7FFFFFFFFFFE3FFF2D
:10247000FFFFFFFC0FFFFFFFFFF00FFFFFFFFFF06D
:102480003FFFFFFFFFFC7FFFFF803FFE7FFFFF005E
:102490003FFEFFFFFE007FFFFFFFFC00FFFFFFFF8F
:1024A000F801FFFFFFFFF003FFFFFFFFE007FFFF63
:1024B000FFFFC007FFFFFFFFC007FFFFFFFFC007D1
:1024C000FFFFFFFFC007FFFFFFFFC007FFFFFFFF8A
:1024D000C007FFE7FFFFC007FFC7FFFFC007FF8779
:1024E000FFFFC007FF07FFFFC007FE07FFFFC00099
:1024F0000007FFFFC0000007FFFFC000000FFFFF45
:102500008000000FFFFF0000001FFFFE0000003FE3
:10251000FFFC0000007FFFF8000000FFFFF000005C
:1025200001FFFFE0000003FFFFC0000007FFFF8086
:10253000007FFFFFFF0000FFFFFFFE0001FFFFFF26
:10254000FC0003FFFFFFF80007FFFFFFF0000FFF95
:10255000FFFFE0001FFFFFFFC3803FFFFFFF87C0BB
:102560007FFFFFFF87C0FFFFFFFF87C1FFFFFFFF68
:102570008383FFFFFFFFC007FFFFFFFFC00FFFFFC9
:10258000FFFF601FFFFFFFFE783FFFFFFFFE3FFFE3
:10259000FFFFFFFC0FFFFFFFFFF00FFFFFFFFFF04C
:1025A0003FFFFFFFFFFC7FFFFFFFFFFE7FC7FFFF37
:1025B000F1FEFF03FFFFE07FFE03FFFFE03FFC03B0
:1025C000FFFFE01FF807F007F00FF00F8000F8079B
:1025D000E01E00003C03E03C00001E03E070000031
:1025E0000703E0E000000383F1C001C001C7FF80E2
:1025F00003E000FFFF8003E000FFFF0003E0007F37
:10260000FF0003E0007FFE0003E0003FFE0003E068
:10261000003FFC0003E0001FFC0003E0001FFC0083
:1026200003E0001FFC0003E0001FFC0003E0001FAC
:10263000FC0003F0001FFC0001F8001FFC0000FC80
:10264000001FFC00003E001FFE00001F003FFE00B8
:10265000000F803FFF000007803FFF000003007F66
:10266000FF80000000FFFF80000000FFFF800000EF
:1026700000FFFF000000007FFE000000003FFC00A4
:102680000000001FFC060000301FFC0F8000F81F38
:10269000FE1FF007FC3FFFFFFFFFFFFFFFFFFFFFF5
:1026A000FFFF7FFFFFFFFFFE7FFFFFFFFFFE3FFFFC
:1026B000FFFFFFFC0FFFFFFFFFF00FFFFFFFFFF02B
:1026C0003FFFFFFFFFFC7FFFF83FFFFE7FFFF01F94
:1026D000FFFEFFFFE38FFFFFFFFFE7CFFFFFFFFFDF
:1026E000E7CFFFFFFFFFE7CFFFFFFFFFE1CFFFFFD8
:1026F000FFFFE1CFFFFFFFFFE7CFFFFFFFFFE7CFC8
:10270000FFFFFFFFE7CFFFFFFFFFE7CFFFFFFFFF69
:10271000E1CFFFFFFFFFE1CFFFFFFFFFE7CFFFFFAD
:10272000FFFFE7CFFFFFFFFFE7CFFFFFFFFFE7CF91
:10273000FFFFFFFFE1CFFFFFFFFFE1CFFFFFFFFF45
:10274000E7CFFFFFFFFFE7CFFFFFFFFFE3CFFFFF75
:10275000FFFFE0CFFFFFFFFFE00FFFFFFFFFE00FF6
:10276000FFFFFFFFE00FFFFFFFFFE00FFFFFFFFF97
:10277000E00FFFFFFFFFE00FFFFFFFFFE00FFFFF96
:10278000FFFFE00FFFFFFFFFC007FFFFFFFF80031A
:10279000FFFFFFFF8003FFFFFFFF8003FFFFFFFF3F
:1027A0008003FFFFFFFF8003FFFFFFFF8003FFFFAA
:1027B000FFFFC007FFFFFFFFC007FFFFFFFFE00FA6
:1027C000FFFF7FFFF01FFFFE7FFFFFFFFFFE3FFFCA
:1027D000FFFFFFFC0FFFFFFFFFF00FFFFFFFFFF00A
:1027E0003FFFFFFFFFFC7FFFFFFFFFFE70003FFF8B
:1027F000FFFEF0001FFFFFFFF0000FFFFFFFF000E4
:1028000007FFFFFFF00003FFFFFFF00001FFFFFFE6
:10281000F00F80FFFFFFF01FC07FFFFFF03FE03FA2
:10282000FFFFF07FF01FFFFFF07FF00FFFFFF07F53
:10283000F007FFFFF07FF003FFFFF03FE001FFFF35
:10284000F03FE000FFFFF01FC0007FFFF00F8000AF
:102850003FFFF80000001FFFFC0000000FFFFE001C
:10286000000007FFFF00000003FFFF80000001FFE2
:10287000FFC0000000FFFFE00000007FFFF000004D
:10288000003FFFF80000001FFFFC0000000FFFFEEC
:1028900000000007FFFF00000003FFFF80000007AB
:1028A000FFFFC000000FFFFFE000001FFFFFF00070
:1028B000003FFFFFF800007FFFFFFC0000FFFFFF6D
:1028C000FE0001FFFFFFFF0003FFFFFFFF8007FF88
:1028D000FFFFFFC00FFFFFFFFFE01FFFFFFFFFF045
:1028E0003FFF7FFFFFF87FFE7FFFFFFCFFFE3FFF04
:1028F000FFFFFFFC0FFFFFFFFFF0000007E01FF8E6
:1029000018181818181800003FFC3C3C3C3C3C3C94
:102910003E7C3E7C3FFC3FFC0000040006000700BC
:102920000F000F801F803F907F187F1C7E3C7C3EF5
:10293000787E78FE31FE11FC09F80FE01FF83FFCAD
:102940007FFEFFE6FFCEFF9FF33FF07FF8FFFDFE27
:102950007FFE7FFC3FF81FF003C000E003C00F00C4
:102960001C3810F003C00F001C3810F003E007E023
:1029700007E00000000003C00380018001800180A7
:10298000199039B8318C618C618660066006600EE2
:10299000700C301C1C780FF003C00380038003C050
:1029A00007C007E00FE00E701E701E701E783FF823
:1029B0003FFC7E7C7E7E7FFE7FFE114082002120D8
:1029C0008FE023FC82004A23E200FE209FF013F8F0
:1029D00080802220C0804221BFF0FBFA8880022044
:1029E0008480022084801A208080E3FE828002019D
:1029F00001000F421FC0784110400840904008423B
:102A00001FC008411040FFFD104008405FC0084053
:102A1000800008413FE00843252010412520104157
:102A200025202041252040417FF07FF8488002008A
:102A300049000201FFF00201001002027F20220083
:102A4000410023F07F00220008002200FF802200C6
:102A500088802200888022008A8022008900FFFC72
:102A6000080023F21FC022111040FBF090402212F8
:102A70001FC02A11104033F1104060005FC0AFFC4E
:102A8000800020413FE02243252022792520224159
:102A90002520A541252048FD7FF01083DFC010824E
:102AA0005040208250402FFFDFC06082520061C240
:102AB0005200A1C25FE022A3D20022A251002492C0
:102AC0005100288E5090308BD45020825830208076
:102AD0001010104047C017FC44402003F44023F876
:102AE00044406208C440A3F8E440200154402FFD54
:102AF00044402806444023F84440204044502040AD
:102B00004850214050302080400020921FC03DF9A5
:102B100090402090904040901FC07BFF0000A0019B
:102B20003FE021F90200FD09020021097FF021F9AF
:102B30000500210945002909888031F91070210814
:102B4000202025004300202070F8360131012B01A0
:102B500023011C01150110010A010301FC00F20010
:102B6000EB00E400E000DB00D300CD00C700C200B2
:102B7000BC00B800B200AD00A600A2009E00980004
:102B8000940091008E008A008700840081007E00FE
:102B900072006D0068003E0053656C6563742054DC
:102BA00069700000000000003E5B4F5B3E3E6B4FD3
:102BB0006B3E1C3E7C3E1C183C7E3C181C577D57CF
:102BC0001C1C5E7F5E1C00183C1800FFE7C3E7FF7B
:102BD0000018241800FFE7DBE7FF30483A060E260E
:102BE00029792926407F050507407F05253F5A3C66
:102BF000E73C5A7F3E1C1C08081C1C3E7F14227FA9
:102C000022145F5F005F5F06097F017F0066899580
:102C10006A606060606094A2FFA29408047E040869
:102C200010207E201008082A1C08081C2A08081EEC
:102C3000101010100C1E0C1E0C30383E3830060ED2
:102C40003E0E06000000000000005F0000000700CC
:102C50000700147F147F14242A7F2A122313086488
:102C60006236495620500008070300001C2241002C
:102C70000041221C002A1C7F1C2A08083E0808006C
:102C8000807030000808080808000060600020100C
:102C90000804023E5149453E00427F4000724949C6
:102CA00049462141494D331814127F1027454545A7
:102CB000393C4A49493141211109073649494936C8
:102CC000464949291E00001400000040340000005D
:102CD000081422411414141414004122140802018F
:102CE0005909063E415D594E7C1211127C7F4949BB
:102CF00049363E414141227F4141413E7F49494958
:102D0000417F090909013E414151737F0808087F4D
:102D100000417F41002040413F017F081422417F54
:102D2000404040407F021C027F7F0408107F3E41EC
:102D300041413E7F090909063E4151215E7F091943
:102D40002946264949493203017F01033F4040405B
:102D50003F1F2040201F3F4038403F63140814634A
:102D600003047804036159494D43007F4141410206
:102D700004081020004141417F0402010204404048
:102D8000404040000307080020545478407F284406
:102D900044383844444428384444287F38545454F0
:102DA0001800087E090218A4A49C787F08040478FF
:102DB00000447D40002040403D007F10284400003A
:102DC000417F40007C047804787C0804047838440F
:102DD000444438FC1824241818242418FC7C0804C3
:102DE0000408485454542404043F44243C404020E4
:102DF0007C1C2040201C3C4030403C44281028448F
:102E00004C9090907C4464544C440008364100003F
:102E100000770000004136080002010204023C264F
:102E200023263C1EA1A161123A4040207A38545416
:102E3000555921555579412154547841215554789B
:102E40004020545579400C1E52721239555555592F
:102E5000395454545939555454580000457C410054
:102E600002457D420001457C40F0292429F0F028EC
:102E70002528F07C545545002054547C547C0A0984
:102E80007F4932494949323248484832324A4848F3
:102E9000303A4141217A3A42402078009DA0A07DFD
:102EA00039444444393D4040403D3C24FF242448BB
:102EB0007E4943662B2FFC2F2BFF0929F620C08863
:102EC0007E090320545479410000447D4130484834
:102ED0004A32384040227A007A0A0A727D0D19314E
:102EE0007D2629292F28262929292630484D4020AA
:102EF000380808080808080808382F10C8ACBA2F86
:102F0000102834FA00007B000008142A142222142E
:102F10002A14089500220095AA005500AAAA55AACD
:102F200055AA000000FF00101010FF00141414FF39
:102F3000001010FF00FF1010F010F0141414FC002B
:102F40001414F700FF0000FF00FF1414F404FC1435
:102F50001417101F10101F101F1414141F0010102E
:102F600010F0000000001F101010101F10101010A3
:102F7000F010000000FF101010101010101010FFC3
:102F800010000000FF140000FF00FF00001F1017DA
:102F90000000FC04F414141710171414F404F400C3
:102FA00000FF00F714141414141414F700F7141489
:102FB00014171410101F101F141414F4141010F010
:102FC00010F000001F101F0000001F14000000FC84
:102FD000140000F010F01010FF10FF141414FF1470
:102FE0001010101F00000000F010FFFFFFFFFFF0A7
:102FF000F0F0F0F0FFFFFF0000000000FFFF0F0FF8
:103000000F0F0F38444438447C2A2A3E147E0202B3
:103010000606027E027E0263554941633844443C01
:1030200004407E201E2006027E020299A5E7A59993
:103030001C2A492A1C4C7201724C304A4D4D3030CA
:1030400048784830BC625A463D3E494949007E01B5
:1030500001017E2A2A2A2A2A44445F444440514AD4
:10306000444040444A51400000FF0103E080FF001B
:103070000008086B6B083612362436060F090F0657
:10308000000018180000001010003040FF0101007F
:103090001F01011E00191D1712003C3C3C3C0000A2
:1030A00000000000000000240027002A00000000AB
:1030B00000250028002B0000000000230026002926
:1030C00000040404040404040402020202020203D1
:1030D00003030303030102040810204080010204DB
:1030E000081020010204081020AED5F0A83FD3003C
:1030F000408D14A1C8DA1281CFD9F1DB40A4A6AF6C
:10310000200021007F220007506C656173652077E5
:10311000616974004144433A200074656D703A203F
:1031200000536574206D6561737572656400537436
:1031300065703A2000FFFFFFFFFFFF80038670806D
:10314000038003867080039FF3E1309FF39FF3E1D8
:10315000309FF3983301CC9833983301CC9833984F
:103160003387C098339833E1C098339833E1C098DF
:10317000339FF398C09FF39FF398C09FF38003663B
:10318000CC8003800366CC8003FFFF010CFFFFFFB0
:10319000FF01001FFF810061301F3F873CE6FC8775
:1031A00033873CE6FC87F3F8039E0F1F03F8039E6A
:1031B0000F1F03E13CFE0C07CFE13CFE0C07CF994B
:1031C000033E3086C3E6CF380F9EF3E6CF380F9E1E
:1031D000F39E0327CC81039E0327CC8103E0FFE10C
:1031E0000CE6CFE0FFE10CE6CF9803060000FF9865
:1031F00003060000FFFFFF1EF0F80380036630990E
:10320000C38003663099C39FF3010CF8FF9FF3015D
:103210000CF8FF9833393C01CF9833393C01CF98F3
:1032200033FF0C793F98333ECCE0F398333ECCE04B
:10323000F39FF33E0098CF9FF33E0098CF80033E6C
:1032400030E7C380033E30E7C3FFFFFFFFFFFFFF10
:10325000FFFFFFFFFF3030300076312E364C31005B
:1032600056005600430000800080018001800380EA
:10327000078007F00FF00FE01FC001C00180018040
:10328000018001000100124812481FF8E0072E14C7
:103290002C04E80720042004E00720042814E00799
:1032A0001FF8124812484552524F5200484F4C44A2
:1032B000004845415400574F524B5900424F4F531D
:1032C0005400534C454550004F46460000007E00D8
:1032D0007F00738061C061E073F03FF81FFC0FFE58
:1032E00007FF03FF01FE00FC007800300102040824
:1032F00010204080000000080002010000030407C5
:103300000000000000000000BA2E5D3811241FBE2E
:10331000CFEFD8E0DEBFCDBF12E0A0E0B1E0E6EC39
:10332000FBE702C005900D92A237B107D9F727E05D
:10333000A2E7B2E001C01D92A43CB207E1F719E197
:10334000C5E8D9E104C02197FE010E94D93BC438E9
:10335000D107C9F70E947E2F0C94D63D0C94000033
:103360004F925F926F927F928F929F92AF92BF9295
:10337000CF92DF92EF92FF920F931F93CF93DF9341
:1033800000D000D0CDB7DEB74B015C0129013A0176
:103390006701780120E030E0A9010E94DE3887FD56
:1033A000A6C020E030E0A901C301B2010E94DE38CE
:1033B00087FD9DC020E030E0A901C801B6010E9450
:1033C000DE3887FD94C081E0209184073091850725
:1033D0002130310509F080E08093A50780926A07CB
:1033E00090926B07A0926C07B0926D0740926E07A7
:1033F00050926F076092700770927107C0927207C7
:10340000D0927307E0927407F09275076091980765
:103410007091990780919A0790919B070E94E338D9
:1034200020E030E04AE754E40E94173B69837A8346
:103430008B839C838092760790927707A09278077F
:10344000B09279079B01AC01C301B2010E944439DB
:103450002B013C0140927A0750927B0760927C07D7
:1034600070927D0729813A814B815C81C701B60149
:103470000E94173B6B017C01C0927E07D0927F07B0
:10348000E0928007F09281078091820790918307F4
:10349000019769F5A501940160E070E0CB010E94FD
:1034A000AA3A609376077093770780937807909392
:1034B0007907A301920160E070E0CB010E94AA3A73
:1034C00060937A0770937B0780937C0790937D07C6
:1034D000A701960160E070E0CB010E94AA3A6093D8
:1034E0007E0770937F0780938007909381070F90EA
:1034F0000F900F900F90DF91CF911F910F91FF9040
:10350000EF90DF90CF90BF90AF909F908F907F9083
:103510006F905F904F90089580389105B0F46034BB
:10352000710598F4ECEEF2E390E1969FD001A0785B
:103530001124A80F6770E60FF11D9491AF53BD4F92
:10354000442321F08C91982B9C93089590958C9115
:103550009823FACFDF92EF92FF920F931F93CF93AE
:10356000DF937C01EB01D22E8B01040F111DC801EA
:103570000134110514F080E490E0C817D9073CF439
:103580004D2DBE01C7010E948C1A2196F0CFDF910C
:10359000CF911F910F91FF90EF90DF900895CF9200
:1035A000DF92EF92FF920F931F93CF93DF936B0104
:1035B000122FEC017C01E40EF11CCE15DF0544F462
:1035C000202F412FB601CE010E94AA1A2196F5CFD5
:1035D000DF91CF911F910F91FF90EF90DF90CF90EF
:1035E00008952F923F924F925F926F927F928F92A7
:1035F0009F92AF92BF92CF92DF92EF92FF920F9382
:103600001F93CF93DF9300D01F92CDB7DEB7C22EAA
:10361000D12C9601280F391F37FD4FC080389105F6
:103620000CF04BC0E9824A017B013C01402E512C39
:10363000160127E0220E311C93E0359427949A95C9
:10364000E1F78B01B12CA12C1B821A82EA81FB814C
:1036500083E0F595E7958A95E1F7EA0DFB1DE80D06
:10366000F91DE4918A819B818770992720E830E0D9
:1036700002C0359527958A95E2F7C901F0E0E2236B
:10368000F923EF2B41F04981B8018A819B81860D96
:10369000971D0E948C1A8A819B8101969B838A8345
:1036A0008C159D059CF2A20CB31C0F5F1F4FC80127
:1036B0008E199F09841595053CF20F900F900F907D
:1036C000DF91CF911F910F91FF90EF90DF90CF90FE
:1036D000BF90AF909F908F907F906F905F904F9032
:1036E0003F902F90089580E0E1ECF2E081118FEFA0
:1036F000002481938193819381930394D1F7ECEA21
:10370000F7E0178616861586148608950895AF92F9
:10371000BF92CF92DF92EF92FF920F931F93CF93BE
:10372000DF936C017B018B01040F151FEB015E0120
:10373000AE18BF08C017D10759F06991D601ED91B5
:10374000FC910190F081E02DC6010995892B79F754
:10375000C501DF91CF911F910F91FF90EF90DF9006
:10376000CF90BF90AF900895FC01538D448D252FCD
:1037700030E0842F90E0821B930B541710F0CF960B
:10378000089501970895FC01918D828D981761F03D
:10379000A28DAE0FBF2FB11D5D968C91928D9F5F54
:1037A0009F73928F90E008958FEF9FEF0895FC0133
:1037B000918D828D981731F0828DE80FF11D858DE6
:1037C00090E008958FEF9FEF0895FC01918D228D79
:1037D000892F90E0805C9F4F821B91098F739927FE
:1037E000089581EC96E00E94E51B21E0892B09F405
:1037F00020E0822F089580E090E0892B29F00E943C
:10380000F11B81110C9400000895FC01A48DA80FF8
:10381000B92FB11DA35ABF4F2C91848D90E0019612
:103820008F739927848FA689B7892C93A089B18932
:103830008C91837080648C93938D848D981306C0D3
:103840000288F389E02D80818F7D80830895EF9237
:10385000FF920F931F93CF93DF93EC0181E0888F4A
:103860009B8D8C8D98131AC0E889F989808185FF1A
:1038700015C09FB7F894EE89FF896083E889F989BC
:1038800080818370806480839FBF81E090E0DF91BE
:10389000CF911F910F91FF90EF900895F62E0B8D11
:1038A00010E00F5F1F4F0F731127E02E8C8D8E11CC
:1038B0000CC00FB607FCFACFE889F989808185FF33
:1038C000F5CFCE010E94051CF1CFEB8DEC0FFD2F43
:1038D000F11DE35AFF4FF0829FB7F8940B8FEA89EE
:1038E000FB8980818062CFCFCF93DF93EC01888DFD
:1038F0008823B9F0AA89BB89E889F9898C9185FD6B
:1039000003C0808186FD0DC00FB607FCF7CF8C91F8
:1039100085FFF2CF808185FFEDCFCE010E94051C8F
:10392000E9CFDF91CF910895833081F028F4813081
:1039300099F08230A9F008958730A9F08830C9F055
:103940008430B1F4809180008F7D03C0809180002D
:103950008F7780938000089584B58F7784BD089514
:1039600084B58F7DFBCF8091B0008F778093B000BE
:1039700008958091B0008F7DF9CFCF93DF93282FEA
:1039800030E0F901EC50FD4C8491F901EB52FF4C11
:10399000D491F901EF53FF4CC491CC23A1F08111D4
:1039A0000E94941CEC2FF0E0EE0FFF1FE954FF4C37
:1039B000A591B491EC91ED2381E090E009F480E0D1
:1039C000DF91CF91089580E090E0FACF1F93CF93DD
:1039D000DF93282F30E0F901EC50FD4C8491F90180
:1039E000EB52FF4CD491F901EF53FF4CC491CC231F
:1039F000A9F0162F81110E94941CEC2FF0E0EE0F1D
:103A0000FF1FE355FF4CA591B4918FB7F894EC914B
:103A1000111108C0D095DE23DC938FBFDF91CF91C9
:103A20001F910895DE2BF8CFCF93DF9390E0FC0138
:103A3000EB52FF4C24918F539F4CFC0184918823BF
:103A4000C9F090E0880F991FFC01ED55FF4CA5913E
:103A5000B491FC01E355FF4CC591D49161110DC0A7
:103A60009FB7F8948C91209582238C93888128238A
:103A700028839FBFDF91CF910895623051F49FB7A3
:103A8000F8943C91822F809583238C93E8812E2B90
:103A9000EFCF8FB7F894EC912E2B2C938FBFEACFFA
:103AA000CF93DF93EC0161E089E00E94141D209721
:103AB00031F460E089E0DF91CF910C94E61CCF3FB8
:103AC000D10511F461E0F6CFEDEFF2E3E491E330DC
:103AD00029F140F4E130B1F0E230D9F0C038D1053D
:103AE0008CF7E7CFE73021F1E83051F1E430B1F75E
:103AF00080918000806280938000D0938B00C0937F
:103B00008A0004C084B5806884BDC7BDDF91CF91B1
:103B1000089584B5806284BDC8BDF8CF80918000CF
:103B2000806880938000D0938900C0938800EECF96
:103B30008091B00080688093B000C093B300E6CF5E
:103B40008091B00080628093B000C093B400DECF5B
:103B50003FB7F89480918B0290918C02A0918D02D6
:103B6000B0918E0226B5A89B05C02F3F19F0019693
:103B7000A11DB11D3FBFBA2FA92F982F8827BC01C7
:103B8000CD01620F711D811D911D42E0660F771FEF
:103B9000881F991F4A95D1F708958F929F92AF92EF
:103BA000BF92CF92DF92EF92FF924B015C010E9495
:103BB000A81D6B017C010E94A81D6C197D098E094E
:103BC0009F09683E734081059105A8F321E0821AA0
:103BD0009108A108B10888EEC80E83E0D81EE11C48
:103BE000F11C81149104A104B10429F7FF90EF9016
:103BF000DF90CF90BF90AF909F908F9008952FB798
:103C0000F894609187027091880280918902909166
:103C10008A022FBF089584E98093BC008091BC0084
:103C200084FDFCCF08958093BB0084E88093BC00A2
:103C30008091BC0087FFFCCF089584EA8093BC008C
:103C40008091BC0087FFFCCF88E70C94131E0E9474
:103C50001D1E80E48093BB0084E88093BC00E1ECEF
:103C6000F2E09091BC0097FFFCCF91919093BB0044
:103C70008093BC0096E0E13CF90799F78091BC0085
:103C800087FFFCCF0C940B1ECF93C82F0E941D1EE4
:103C900080E00E94131E8C2F0E94131ECF910C9463
:103CA0000B1E480F592F511D4138510514F040E8A3
:103CB00050E0481BFB0177FD379633E0F595E7951B
:103CC0003A95E1F7F695FE2FEE27F795E795E80F81
:103CD000F91FEF53FD4F6770772781E090E001C037
:103CE000880F6A95EAF7382F213041F4415078F077
:103CF0008191DF011197832B8C93F8CF80954150F0
:103D000030F09191DF01119798239C93F8CF08959B
:103D1000CF92DF92EF92FF920F93CF93DF936C01DC
:103D20007B01C42FD22F202F0E94511EB7016D0F8F
:103D3000711D61507109603471052CF4202F4C2FD6
:103D4000C6010E94511E202F4D2FB701C6010E94AF
:103D5000AA1AC6018C0F911D202F4D2FB701019774
:103D6000DF91CF910F91FF90EF90DF90CF900C9467
:103D7000AA1A2F923F924F925F926F927F928F92E8
:103D80009F92AF92BF92CF92DF92EF92FF920F93EA
:103D90001F93CF93DF93CDB7DEB72A970FB6F89472
:103DA000DEBF0FBECDBF9A8389836A3061F5DC0127
:103DB00052968C91B8E08B9F90011124E981FA8191
:103DC00086859785820F931F978786871586148629
:103DD00081E090E02A960FB6F894DEBF0FBECDBF0B
:103DE000DF91CF911F910F91FF90EF90DF90CF90D7
:103DF000BF90AF909F908F907F906F905F904F900B
:103E00003F902F9008956D3019F329813A813A87B8
:103E10002987D9011C96AD90BC90B0E8AB16B104CF
:103E20000CF07BC0F901C684D784F0E4CF16D1042E
:103E30000CF073C0D90152966C90529745E09501F1
:103E4000649E200D311D1124121613060CF065C05E
:103E5000262C312C910153E0220F331F5A95E1F7A4
:103E60002C0D3D1D121613060CF057C05196BC9137
:103E7000BB83E985FA85F089FC83649FB001112436
:103E80009B012D55344D3A832983712CE981FA81A8
:103E90008491F5E07F1201C080E0460138E0532EA6
:103EA000282F30E03E832D834C8080FF4B804110D3
:103EB00004C03B818C813817E1F010E000E006156A
:103EC000C0F4D501A00FB11FB887AF83F12CE12C4E
:103ED000E61460F4B701680D791D442D8F81988533
:103EE0000E948C1ABFEFEB1AFB0AF2CF0F5F1F4F35
:103EF000E6CF8D819E81959587955A94820C931C6F
:103F00005110CECF7394E981FA813196FA83E98317
:103F1000A20CB31CF6E07F12B9CFA985BA855296E0
:103F20002C915297422F50E01C968D919C91B6E0B7
:103F30002B9F800D911D1124E985FA859587848733
:103F40002389222309F444CF6AEF64039001659F1B
:103F5000300D112420583F4F281739070CF038CF67
:103F6000DF010190F081E02D0190F081E02D6AE009
:103F7000CD0109952DCF0F931F93CF93DF938C0124
:103F8000D0E0C0E0F801EC0FFD1F6491662341F022
:103F90008CEA97E00E94B91E892B11F02196F2CF8E
:103FA000CE01DF91CF911F910F910895682F8CEA78
:103FB00097E00C94B91E90E080E0089580917A001B
:103FC000806980937A008EE480937C0061E070E0E9
:103FD00080E090E00E94CD1D83B7817F826083BF27
:103FE00080E130E020E093B7916093BF889593B76C
:103FF0009E7F93BF90917A0096FDFCCF4091780010
:1040000050917900240F351F815069F780917A0013
:104010008F7780937A0084E0369527958A95E1F72B
:1040200050E040E064EB7BE281E190E00E94183ACE
:10403000C901089580917A00806980937A0088ECA4
:1040400080937C0064E170E080E090E00E94CD1DF0
:1040500083B7817F826083BF80E270E060E093B7C6
:10406000916093BF889593B79E7F93BF90917A009C
:1040700096FDFCCF2091780030917900620F731F7C
:10408000815069F780917A008F7780937A007695D6
:1040900067957695679562527A4090E080E00E943D
:1040A000E33826EF38E24CE151E40E94173B0895D3
:1040B00090917A00906990937A008E5080648093FA
:1040C0007C0083B7817F826083BF20E290E080E044
:1040D00033B7316033BF889533B73E7F33BF3091FC
:1040E0007A0036FDFCCF4091780050917900840F22
:1040F000951F215069F720917A002F7720937A003D
:1041000025E0969587952A95E1F708958FE00E941E
:104110005820A0919202B09193029C010E949B3A78
:104120000E94E53828E539E743E353E40E94173B52
:104130000E94903BCB0108952091A00230E0EEE177
:10414000F2E090E080E0AF014E5152404217530739
:1041500024F44191840F911DF6CF08958091990226
:10416000882369F086E00E94BD1C892B41F06AE03B
:1041700070E080E090E00E94CD1D109299020895B9
:104180000F931F93CF9380914801882399F0CFEF2D
:104190000FEE11E061E085E00E94E61CC801019786
:1041A000F1F760E085E00E94E61CC8010197F1F795
:1041B000C15081F7CF911F910F9108952F923F9297
:1041C0004F925F926F927F928F929F92AF92BF9227
:1041D000CF92DF92EF92FF920F931F93CF93DF93D3
:1041E00010E000E0D0E0C0E03EE3E32EF12C40EC34
:1041F000C42ED12CAA24A394B12C60E2662E712C7B
:1042000070E4272E312C4C2E86E00E94BD1C21E04C
:10421000892B09F020E020939902F0929F02E0920E
:104220009E02D0929D02C0929C02B0929B02A092EC
:104230009A0282E890E09093AB028093AA02809168
:10424000AA029091AB0295958795582E9FE159123D
:1042500043C0F0929F02E0929E02D0929D02C092D3
:104260009C02B0929B02A0929A02EEEBF0E0F093D7
:10427000AB02E093AA029FE5592E0E94731B82E0D5
:104280008093BE071093B9070093B807E0E3F0E00E
:10429000F093BB07E093BA078EE50E94D61F1092F9
:1042A000B9071092B8077092BB076092BA07912CB9
:1042B000812C841438F58091BD02F40196E0989F1A
:1042C000E00DF11D1124E05BFE4F80810E94D61F9E
:1042D000EFEF8E1A9E0AEDCFF0E65F12CECFF0928E
:1042E0009F02E0929E02D0929D02C0929C02B092E8
:1042F0009B02A0929A023092AB022092AA0280E224
:10430000582EBBCF1093B9070093B8077092BB0724
:104310006092BA07852D0E94D61F0E94AE200E948F
:10432000271E86E00E94BD1C892B09F088CF809152
:104330009902811184CF8090BD02F6E08F9E4001EA
:104340001124C401805B9E4F4C01FC01EC0FFD1F4A
:1043500050820E94C0206AE070E080E090E00E94FD
:10436000CD1D2196005F1F4FC530D10509F04BCF01
:10437000F4011582DF91CF911F910F91FF90EF9083
:10438000DF90CF90BF90AF909F908F907F906F9075
:104390005F904F903F902F9008953F924F925F9281
:1043A0006F927F928F929F92AF92BF92CF92DF9245
:1043B000EF92FF920F931F93CF93DF93CDB7DEB7AA
:1043C0002E970FB6F894DEBF0FBECDBF8091BC0212
:1043D000882309F4A5C110925E0710925F0710921E
:1043E00060071092610780905E0790905F07A09031
:1043F0006007B0906107C090B302D090B402E09023
:10440000B502F090B602A7019601C501B4010E9461
:10441000AA3A2B013C0120E030E0A9010E94BF3BF9
:1044200018160CF0A0C1C301B2010E94903B80910C
:104430004901882309F4B8C1C0926607D092670782
:10444000E0926807F0926907E12CF12C00EA10E491
:1044500020E030E040E450E46E31710540F0E12CA2
:10446000F12C00E81FE320E030E040E05FE360E093
:1044700070E080E391E40E94B0198091A407882342
:1044800009F42AC10E94FF1D6D837E838F83988764
:1044900080918C0790918D07A0918E07B0918F0726
:1044A0004D815E816F817885481B590B6A0B7B0BB0
:1044B0008091980790919907A0919A07B0919B07D6
:1044C000481759076A077B0708F406C1E091860779
:1044D000F091870780819181A281B38189839A833A
:1044E000AB83BC83E0918A07F0918B079C01AD01FF
:1044F00060817181828193810E94AA3A4B015C01A3
:104500002091940730919507409196075091970715
:1045100069817A818B819C810E94AA3A6B017C011E
:1045200020917A0730917B0740917C0750917D075D
:10453000C501B4010E944439209190073091910740
:1045400040919207509193070E94AB3A2B013C0196
:104550004092900750929107609292077092930751
:104560003090A50731101AC0209176073091770757
:104570004091780750917907C701B6010E944439EC
:104580009B01AC01C301B2010E94AA3A609390075B
:1045900070939107809392079093930740909007B0
:1045A0005090910760909207709093071091A00728
:1045B0009091A1079E87A091A207AD870091A307C4
:1045C000212F392F4A2F502FC301B2010E94BF3B28
:1045D00018160CF0CCC0812F9E85AD85B02F80932E
:1045E000900790939107A0939207B093930733207D
:1045F00009F4D6C02091760730917707409178076B
:1046000050917907C501B4010E9444394B015C0106
:1046100020917E0730917F0740918007509181075C
:10462000C701B6010E9444399B01AC01609190071B
:104630007091910780919207909193070E94AA3AF6
:10464000A50194010E94AB3A6B017C019B01AC0176
:10465000612F7E858D85902F0E94DE3887FD18C0E2
:1046600010919C0790919D079E87A0919E07AD8712
:1046700000919F07212F392F4A2F502FB601C701D4
:104680000E94DE3887FD04C01C2DDE86ED860F2DCE
:10469000E0918807F0918907812F9E85AD85B02F25
:1046A00080839183A283B38389819A81AB81BC810A
:1046B0008093940790939507A0939607B0939707DC
:1046C0008D819E81AF81B88580938C0790938D07F3
:1046D000A0938E07B0938F07609162077091630774
:1046E00080916407909165070E94893BCB012E96CB
:1046F0000FB6F894DEBF0FBECDBFDF91CF911F91F3
:104700000F91FF90EF90DF90CF90BF90AF909F9070
:104710008F907F906F905F904F903F900C94501DC2
:104720008091BB02609144017091450181110EC0DE
:104730008091B1029091B2022091BA02BC01222371
:1047400029F060914301680F792F711D90E080E09E
:104750000E94E33860935E0770935F078093600761
:104760009093610740CEC301B20190585ECE809114
:104770009C0790919D07A0919E07B0919F07898704
:104780009A87AB87BC879C01AD01C301B2010E942F
:10479000DE3887FF2CCF89859A85AB85BC851FCFF6
:1047A000812C912C540134CF20E030E040E05FE3D5
:1047B000C701B6010E94AB3A9B01AC01C501B4012F
:1047C0000E94BF3B18164CF41092620710926307C8
:1047D00010926407109265077FCF80E090E0AFE70A
:1047E000B3E48093620790936307A0936407B09348
:1047F000650772CF4F925F926F927F928F929F92D6
:10480000AF92BF92CF92DF92EF92FF92CF93DF935E
:104810008090940290909502A0909602B09097029A
:10482000C091BD02D0E0C501B4010E94893B6B017B
:104830007C0120E030E048E453E4C501B4010E946B
:10484000DE3893E0CC0FDD1F9A95E1F7CE5FDE4FA7
:1048500087FF31C02881398150E040E0255131097E
:1048600041095109C701B6010E94C93B28EC30E05B
:1048700040E050E00E94183ACA01B9016B5E7F4FD8
:104880008F4F9F4F0E94E5386093B3027093B4023C
:104890008093B5029093B602DF91CF91FF90EF9095
:1048A000DF90CF90BF90AF909F908F907F906F9050
:1048B0005F904F9008954A805B80712C612C20E0BE
:1048C00030E04CE853E4C501B4010E94DE3887FFB4
:1048D0001FC088809980B12CA12CA7019601285C6B
:1048E000310941095109C301B201681979098A09DD
:1048F0009B090E94C93B20E530E040E050E00E9467
:10490000183ACA01B901680D791D8A1D9B1DBACFDD
:104910002C813D8150E040E02419350946095709B2
:10492000C701B60168517140810991090E94C93BD4
:1049300020E530E040E050E00E94183ACA01B90199
:10494000640D751D861D971D9DCFFC0101900020F3
:10495000E9F73197AF01481B590BBC018CEA97E08E
:104960000C94871B8F929F92AF92BF920F931F93CD
:10497000CF93DF93CDB7DEB7A1970FB6F894DEBF24
:104980000FBECDBF19A2423008F44AE08E010F5D80
:104990001F4F842E912CB12CA12CA50194010E94B3
:1049A000793AE62FB901CA01EA30F4F4E05DD801A2
:1049B000EE938D01232B242B252B79F790E080E0BB
:1049C000109719F0CD010E94A524A1960FB6F89476
:1049D000DEBF0FBECDBFDF91CF911F910F91BF9072
:1049E000AF909F908F900895E95CE1CFCF92DF92D6
:1049F000EF92FF92CF93DF9397FF19C06B017C0179
:104A00008DE20E94D61FEC0166277727CB016C1937
:104A10007D098E099F094AE00E94B2248C0F9D1FD8
:104A2000DF91CF91FF90EF90DF90CF9008954AE013
:104A3000DF91CF91FF90EF90DF90CF900C94B22454
:104A40004F925F926F927F928F929F92AF92BF929E
:104A5000CF92DF92EF92FF920F931F93CF936B0150
:104A60007C01742EAC019B010E94C43B882399F009
:104A700083E692E0CF911F910F91FF90EF90DF902E
:104A8000CF90BF90AF909F908F907F906F905F90EE
:104A90004F900C94A52446015701E894B7F82FEFE6
:104AA0003FEF4FE75FE7C501B4010E94C43B8111AE
:104AB0000DC02FEF3FEF4FE75FE7C501B4010E9444
:104AC000DE3818161CF487E692E0D4CF2FEF3FEFC4
:104AD0004FE75FE4C701B6010E94BF3B18161CF404
:104AE0008BE692E0C7CF2FEF3FEF4FE75FECC701B8
:104AF000B6010E94DE3887FDF3CF20E030E0A90147
:104B0000C701B6010E94DE3810E000E087FF08C050
:104B10008DE20E94D61F8C01F7FAF094F7F8F0941A
:104B2000C0E060E070E080E09FE37C1641F020E0B0
:104B300030E040E251E40E94173BCF5FF6CFA7017F
:104B400096010E94AB3A2B013C010E94903B4B0125
:104B50005C014AE00E94B2247C01E00EF11ECC23ED
:104B6000B1F1C501B4010E94E3389B01AC01C3015E
:104B7000B2010E94AA3A4B015C018EE20E94D61F4C
:104B8000E80EF91EC15018F120E030E040E251E497
:104B9000C501B4010E9444392B013C010E94903BA5
:104BA0004B01B12CA12C4AE0C501B4010E94B224F2
:104BB000E80EF91EC501B4010E94E3389B01AC0167
:104BC000C301B2010E94AA3A4B015C01DBCFC701CD
:104BD000CF911F910F91FF90EF90DF90CF90BF90FA
:104BE000AF909F908F907F906F905F904F900895BF
:104BF000CF92DF92EF92FF920F931F93CF93DF93A9
:104C0000C82F81E0DC2FD827D093BD07C093BC0705
:104C10008093BE070C2F2EE046E661E370E081E052
:104C200090E00E94881E2091BE023091BF02253F75
:104C300081E03807B8F4A4E6B0E00E949B3A24EF84
:104C400031E040E050E00E94183ABA01A9014E5FFD
:104C50005F4F6F4F7F4F2EE061E370E081E090E0A7
:104C60000E94CF1A60915E0770915F078091600784
:104C7000909161070E94893B9B01AC01A4E6B0E0E2
:104C80000E94373A34EFC32EDD24D394E12CF12C6B
:104C9000A70196010E94183ADA01C9010296A11DE6
:104CA000B11D02970C2F2DE043E062E370E00E94FB
:104CB000CF1A60915E0770915F07809160079091B5
:104CC00061070E94893B9B01AC01A4E6B0E00E9411
:104CD000373AA70196010E94183ADA01C9010296F3
:104CE000A11DB11D039724E045E06CE370E00E9434
:104CF000CF1A60915E0770915F0780916007909175
:104D000061070E94893B9B01AC01A4E6B0E00E94D0
:104D1000373AA70196010E94183A89019A010E5F5D
:104D20001F4F2F4F3F4F0150110941E3E42EF12C4B
:104D30004D2FB701C8010E948C1A8FEFE81AF80AAC
:104D40008DE3E816F104A1F760915E0770915F07AB
:104D500080916007909161070E94893B9B01AC01A3
:104D6000A4E6B0E00E94373A24EF31E040E050E0A2
:104D70000E94183ADA01C9010296A11DB11D0397DC
:104D8000ED2E04E025E046E45BE26BE370E00E9478
:104D9000F11A0C2F2EE047E161E370E088E690E025
:104DA0000E94881E6091620770916307809164077A
:104DB000909165070E94893B9B01AC012F5F3109EF
:104DC00041095109A7E1B0E00E94373ACC24C394CD
:104DD000DD24DA94ED2CFD2CA70196010E94183AEF
:104DE000422F2EE061E370E088E690E00E94CF1A47
:104DF000C093BD07D093BC0782E090E09093B907C1
:104E00008093B80707E310E01093BB070093BA073D
:104E100060915E0770915F078091600790916107D4
:104E200040E00E94202588EF0E94D61F84E49BE288
:104E30000E94BB1F89E690E09093B9078093B80762
:104E40001093BB070093BA076091620770916307E4
:104E500080916407909165070E94893B9B01AC019A
:104E60002F5F310941095109A4E6B0E00E94373AA9
:104E7000A70196010E94183ACA01B9010E94F624BE
:104E800082E49BE20E94BB1FD093BD07C093BC0786
:104E9000DF91CF911F910F91FF90EF90DF90CF9016
:104EA00008956F927F928F929F92AF92BF92CF920E
:104EB000DF92EF92FF920F931F93CF93DF93B09007
:104EC000BD0277247394B11001C0712C809142010E
:104ED0008150990B10929F0210929E02880F991F89
:104EE00090939D0280939C0281E090E090939B02BE
:104EF00080939A028B2D90E0880F991F9093AB02BC
:104F00008093AA0286E00E94BD1C21E0892B09F053
:104F100020E020939902FF24F39472E0972EE6E0BC
:104F20008E2EFCE0CF2ED12C0E94731BC091AA02C2
:104F3000D091AB02D595C795EC2E8E011127C801F3
:104F4000870D911D77FC9A958B199109712C97FD0E
:104F500006C08330910514F082E090E0782EF09244
:104F6000BD071092BC079092BE071092B90710922D
:104F7000B8071092BB071092BA0788E99BE20E941B
:104F8000BB1F1092BD07F092BC071092B907109298
:104F9000B807A72C072C000CBB08C501019654E0EC
:104FA000880F991F5A95E1F79093BB078093BA0732
:104FB00086E99BE20E94BB1F6C2E671890E080E0A0
:104FC00098012A193B095901209142018C010F5F78
:104FD0001F4F6216D0F4D092B907C092B80798015B
:104FE00044E0220F331F4A95E1F73093BB0720932B
:104FF000BA078A0D9B1D889E9001899E300D112451
:10500000C901805B9E4F0E94A524C80163940330B0
:105010001105D1F60E94AE200E94271E86E00E9454
:10502000BD1C892BB9F480919902811113C00E9493
:10503000C020E092BD02DF91CF911F910F91FF90B0
:10504000EF90DF90CF90BF90AF909F908F907F9028
:105050006F900895BC2E68CF0E94C13DEF92FF92E1
:105060000F931F93CF93DF93EC017B018A0188811B
:105070009981009729F02A813B812417350788F40C
:10508000B8016F5F7F4F0E94043D009791F09983B4
:1050900088831B830A832C813D81232B11F4FC011F
:1050A00010821D830C83B701888199810E94CF3DB6
:1050B0000CC088819981009711F00E947B3C198275
:1050C00018821D821C821B821A82CE01DF91CF9131
:1050D0001F910F91FF90EF9008951F93CF93DF934F
:1050E000EC01162F0E94023A181739F0612FCE01F9
:1050F000DF91CF911F910C940A3ADF91CF911F91CC
:105100000895AF92BF92CF92DF92EF92FF920F93EA
:105110001F93CF93DF936091470182E090E00E945C
:105120006D286091460183E090E00E946D286091B7
:10513000450184E090E00E946D286091440185E083
:1051400090E00E946D286091430186E090E00E940B
:105150006D2860914C0187E090E00E946D2860917D
:105160004B0188E090E00E946D2860914A0189E03F
:1051700090E00E946D286091C0028AE090E00E9459
:105180006D28609149018BE090E00E946D2860914C
:1051900048018CE090E00E946D286091BD028DE096
:1051A00090E00E946D28609142018EE090E00E94A4
:1051B0006D2860914E018FE090E00E946D28609113
:1051C000980280E190E00E946D2881E1E82EF12CA8
:1051D00010E006E0809142011817B8F5109F6001B9
:1051E0001124D0E0C0E0FE01EC0DFD1DE05BFE4FA0
:1051F0006081C7018C0F9D1F0E946D282196C630CB
:10520000D10589F7670186E0C80ED11C88E0189F98
:10521000E0011124CE5FDE4F8EE0E80EF11C6981C3
:105220002296C6010E946D28560182E0A80EB11C8C
:10523000FE0132976081C60101960E946D286501CA
:10524000AE14BF0461F71F5FC5CFDF91CF911F91EF
:105250000F91FF90EF90DF90CF90BF90AF900895A7
:105260008F929F92AF92BF92CF92DF92EF92FF9276
:10527000CF938FEF90E00E94501D8BEA94E001974E
:10528000F1F78EE00E9458207C018AE00E94BD1C4C
:1052900090917202981729F091E09093B702809351
:1052A0007202809101019FEF980F9093010181118B
:1052B00006C00E9486209093B9028093B802609144
:1052C00062077091630780916407909165070E945F
:1052D000893BCB010E94501D8090940290909502D2
:1052E000A0909602B0909702B70190E080E00E94F3
:1052F000E338A50194010E94AA3A2DEC3CEC4CE461
:105300005DE30E944439A50194010E94AB3A609389
:1053100094027093950280939602909397020E9454
:10532000FA236091BE027091BF0290E080E00E947B
:10533000E3386B017C0120915E0730915F0740915B
:105340006007509161070E94DE388111B5C020913D
:10535000B3023091B4024091B5025091B602C70138
:10536000B6010E94AA3A6B017C0120E030E0A9015D
:105370000E94BF3B18160CF095C020E030E040EAD8
:1053800050E4C701B6010E94BF3B18160CF494C04C
:105390006091B1027091B20290E080E00E94E33827
:1053A0002091B3023091B4024091B5025091B602FF
:1053B0000E94AA3A6B017C0120E030E0A9010E9422
:1053C000BF3B18160CF087C0C701B6010E94903B86
:1053D0006530710508F083C080914F01811105C0CF
:1053E00080914D0181110E94C02081E080934F0186
:1053F00010924D018091BE029091BF02853F21E045
:10540000920710F01092000120910001211140C07C
:10541000843F9140E8F58FEF90E00E94501D0E947C
:10542000C020C1E0C09300010E9451270E94812842
:10543000C093B7028EE00E945820BC0190E080E04B
:105440000E94E338609394027093950280939602D1
:10545000909397021092A9028091B1029091B202AA
:1054600024E630E030939F0220939E0220E233E056
:1054700030939D0220939C022AE030E030939B02FF
:1054800020939A02880F991F9093AB028093AA02EF
:10549000CF91FF90EF90DF90CF90BF90AF909F9013
:1054A0008F90089520E030E040EA50ECC701B6014B
:1054B0000E94DE3887FF6CCF6091B3027091B40216
:1054C0008091B5029091B6020E94903B7093BF020A
:1054D0006093BE025DCFC701B601905877CF10929E
:1054E0004F0188CF0C94023A2F923F924F925F92D5
:1054F0006F927F928F929F92AF92BF92CF92DF92E4
:10550000EF92FF920F931F93CF93DF93CDB7DEB748
:1055100068970FB6F894DEBF0FBECDBF26E020938C
:10552000BE0721E02093BD071092BC070091AA0797
:105530001091AB076091A6077091A70730E8232E62
:1055400032E0332EF10130E020E02017310730F453
:10555000DB01A20FB31F6115710521F410927302D4
:10556000A3E7B2E04C9150E0419351932F5F3F4F3E
:105570002330310551F71C8A1B8A1E8A1D8A188E1A
:105580001F8A4AE08E010F5F1F4FB8010E949438B6
:10559000F80101900020E9F73197AF01401B510B52
:1055A000B801CE0143960E942E288091A6079091C3
:1055B000A707009709F4E8C06B897C89611571051C
:1055C00009F4E0C04091A8075091A9072F89388DB0
:1055D0004217530708F4D6C00E94CF3D8F89988D9B
:1055E0009093AB078093AA07188E1F8A8B899C899A
:1055F000009711F00E947B3C94E7E92E92E0F92E8F
:1056000024E0A22EB12CD12CC12C8091AA0790911C
:10561000AB07C816D90638F4E091A607F091A707A2
:10562000309709F0C8C010927302E3E7F2E080817E
:1056300090E0F10120813181821B930BF2E3F89F0E
:10564000B001F99F700D1124072E000C880B990BE7
:105650000E94E538F70120813181428153810E9407
:10566000AB3A2B013C0120E030E0A9010E94DE387A
:105670008111A4C0F701408251826282738201E0ED
:1056800022E346E270E060E0C50104970E94CF1A71
:105690008EEC882E99249A940FEF1FEFF70120814A
:1056A00031814281538160E070E080E890E40E94A3
:1056B000AA3A2B013C01B401092C000C880B990B70
:1056C0000E94E5389B01AC01C301B2010E94AB3AD4
:1056D0000E94893BB092B907A092B8077093BB07AC
:1056E0006093BA07F10160817181600F711F60538F
:1056F0007109072E000C880B990B0E94F6240F5F8E
:105700001F4FF2E38F0E911C0230110539F62FEF77
:10571000C21AD20A84E0E80EF11CECE2AE0EB11C13
:10572000F2E02F0E311C23E0C216D10409F06DCF38
:1057300000E022E040E870E060E090E080E00E945D
:10574000CF1A2DE040E863E370E090E080E00E9433
:10575000CF1A68960FB6F894DEBF0FBECDBFDF91AB
:10576000CF911F910F91FF90EF90DF90CF90BF905E
:10577000AF909F908F907F906F905F904F903F90F1
:105780002F9008950E947B3C8B899C899093A7075A
:105790008093A6078D899E899093A9078093A80777
:1057A0008F89988D9093AB078093AA071C8A1B8AD8
:1057B0001E8A1D8A19CFEC0DFD1D39CFC301B20120
:1057C00090582DEC3CEC4CE45FE30E944439A3017B
:1057D00092010E94AB3AF7016083718382839383C5
:1057E0004ECF86E00E94BD1C21E0892B09F020E00D
:1057F000209399020E94731B8091AA029091AB02A0
:10580000959587950E94742A0E94271E0E94AE20BB
:1058100086E00E94BD1C892B69F780919902811155
:10582000E9CF0E94C0208091A6079091A70700971A
:1058300021F00E946638CB01089560E070E0CB0152
:10584000FACF2F923F924F925F926F927F928F92F8
:105850009F92AF92BF92CF92DF92EF92FF920F93FF
:105860001F93CF93DF93CDB7DEB72A970FB6F89487
:10587000DEBF0FBECDBF782EE091A002F0E0E25E69
:10588000FD4F80818150990B10929F0210929E02D1
:10589000880F991F90939D0280939C0281E090E075
:1058A00090939B0280939A02872D90E0880F991F16
:1058B0009093AB028093AA0286E00E94BD1C21E077
:1058C000892B09F020E0209399021092BD0781E016
:1058D0008093BC0748E3F42E8090AA029090AB021C
:1058E00095948794182D5401BB24950127193109EB
:1058F000F29EC001F39E900D1124C80ED91EC11452
:10590000D10409F1662777276C197D09072E000C51
:10591000880B990B0E94E53820E030E040E05FE31F
:105920000E9444392B013C01B601DD0C880B990B18
:105930000E94E5389B01AC01C301B2010E94AB3A61
:105940000E94893B6B010E94731B350182E0681A3B
:1059500071082601150193E0290E311C77FC20C047
:10596000E091A002F0E0E25EFD4F80818615170411
:10597000B9F0B4F00E949C20F301E80FF11DEE0F86
:10598000FF1FEE52FE4F40815181EE24E39400E36D
:1059900020E370E060E0C201885491090E94F11A8E
:1059A0008FEF681A780A98E3490E511C6214730449
:1059B000A9F680914E01811140C00E949C20F50102
:1059C000E80FF11DEE0FFF1FEA57FE4F4081518196
:1059D000EE24E39400E124E260E370E080E390E0F1
:1059E0000E94F11A0E94271E0E94AE2086E00E94AB
:1059F000BD1C892B01F58091990281111CC00E9468
:105A0000C020812F2A960FB6F894DEBF0FBECDBFFF
:105A1000DF91CF911F910F91FF90EF90DF90CF908A
:105A2000BF90AF909F908F907F906F905F904F90BE
:105A30003F902F900895782C4FCF80E390E0909383
:105A4000B9078093B80781E390E09093BB078093F8
:105A5000BA0781E08093BE070E949C20880DE82F42
:105A6000F0E0EE0FFF1FE65BF44D65917491CE01FF
:105A700001960E948D38CE0101960E94A524B2CFD6
:105A80001F920F920FB60F9211242F933F934F93B3
:105A90005F936F937F938F939F93AF93BF93EF9396
:105AA000FF9381EC96E00E94051CFF91EF91BF915E
:105AB000AF919F918F917F916F915F914F913F91A6
:105AC0002F910F900FBE0F901F9018951F920F925D
:105AD0000FB60F9211242F938F939F93EF93FF9301
:105AE000E091D106F091D2068081E091D706F09145
:105AF000D80682FD1BC090818091DA068F5F8F737C
:105B00002091DB06821741F0E091DA06F0E0EF53D6
:105B1000F94F958F8093DA06FF91EF919F918F91C6
:105B20002F910F900FBE0F901F9018958081F4CF8A
:105B30001F920F920FB60F9211242F933F938F93C2
:105B40009F93AF93BF938091870290918802A09119
:105B50008902B0918A023091860223E0230F2D370B
:105B600058F50196A11DB11D2093860280938702EE
:105B700090938802A0938902B0938A0280918B024D
:105B800090918C02A0918D02B0918E020196A11D80
:105B9000B11D80938B0290938C02A0938D02B093E1
:105BA0008E02BF91AF919F918F913F912F910F9056
:105BB0000FBE0F901F90189526E8230F0296A11D87
:105BC000B11DD2CF1F920F920FB60F9211242F93B7
:105BD0003F934F935F936F937F938F939F93EF9335
:105BE000FF9383B1817029B190919102981709F4C4
:105BF0009DC030E0220F232F221F330B922F809362
:105C0000910240919002241709F490C020939002D1
:105C100020919A0230919B02981719F031952195A5
:105C200031094091AA025091AB0260919E0270919D
:105C30009F02240F351F261737070CF48BC02091C5
:105C40009A0230919B02981719F0319521953109EC
:105C50004091AA025091AB0260919C0270919D020A
:105C6000240F351F621773070CF46FC040919A021E
:105C700050919B02981719F0519541955109209127
:105C8000AA023091AB02240F351F3093AB02209350
:105C9000AA0241E0981340E020918F02421709F4D4
:105CA00040C020919A0230919B02981719F03195CB
:105CB000219531096091AA027091AB02E0919E0298
:105CC000F0919F02260F371F2E173F070CF44CC090
:105CD00020919A0230919B02981719F031952195E5
:105CE00031096091AA027091AB02E0919C02F0919F
:105CF0009D02260F371FE217F3078CF120919A02BD
:105D000030919B02981719F03195219531098091B6
:105D1000AA029091AB02820F931F9093AB028093E3
:105D2000AA0240938F0281E08093B702FF91EF9126
:105D30009F918F917F916F915F914F913F912F91A3
:105D40000F900FBE0F901F90189520919C023091DC
:105D50009D029BCF20919E0230919F0296CF809111
:105D60009C0290919D02D9CF80919E0290919F02BA
:105D7000D4CF18950F931F93CF93DF93E1ECF6E008
:105D80001382128288EE93E0A0E0B0E084839583D2
:105D9000A683B78389E492E09183808385EC90E0C9
:105DA0009587848784EC90E09787868780EC90E0E5
:105DB000918B808B81EC90E0938B828B82EC90E0D6
:105DC000958B848B86EC90E0978B868B118E128E50
:105DD000138E148EECEAF7E0138212821682178279
:105DE00080E180871582148212868BE592E0918390
:105DF0008083158614861786168611E0108B118A0B
:105E0000128B138AE6EAF7E0118210821382128263
:105E10001582148250E040E061E772E0CF010E94F9
:105E20002E28CAE6D7E082E697E09F8F8E8F86E61F
:105E300097E09D8F8C8F8EE597E099A388A31AAE8B
:105E40001AAA1BAA1CAA1DAA80E090E0AFE7B3E43F
:105E50008EAB9FABA8AFB9AF84E690E0A0E0B0E016
:105E60008EA79FA7A8ABB9AB81E090E0998F888FF0
:105E70009B8F8A8F1BAF80E090E0A0E3B1E4888322
:105E80009983AA83BB8380E090E0A0E0BFE38C838A
:105E90009D83AE83BF8380E090E0A0E8BFE3888766
:105EA0009987AA87BB8780E090E0A0E3B1EC8C875C
:105EB0009D87AE87BF878DEC9CECACE4BDEB888BF7
:105EC000998BAA8BBB8B80E090E0A0E2B1EC8C8B2D
:105ED0009D8BAE8BBF8B0E94FF1D0EA51FA528A911
:105EE00039A9601B710B820B930B6AA37BA38CA354
:105EF0009DA3DF91CF911F910F910895CF93DF93D1
:105F0000CDB7DEB72A970FB6F894DEBF0FBECDBF70
:105F1000789484B5826084BD84B5816084BD85B584
:105F2000826085BD85B5816085BD80916E00816090
:105F300080936E0010928100809181008260809336
:105F40008100809181008160809381008091800038
:105F50008160809380008091B10084608093B10063
:105F60008091B00081608093B00080917A0084605D
:105F700080937A0080917A00826080937A00809189
:105F80007A00816080937A0080917A0080688093A3
:105F90007A001092C1001092B90088E48093B80092
:105FA0000E941D1E80E00E94131E09EE10E388E08F
:105FB000E82E81E3F82EF80184910E94131E0F5FF2
:105FC0001F4FE016F106B9F70E940B1E11E0109367
:105FD000B8000E94271E81E28093B40760E08EE043
:105FE0000E94141D60E08FE00E94141D61E085E0B6
:105FF0000E94141D61E089E00E94141D62E087E0A8
:106000000E94141D62E088E00E94141D62E086E098
:106010000E94141D62E08AE00E94141D8FEF90E040
:106020000E94501D60E085E00E94E61C80917A008D
:10603000876080937A0080917A00886080937A00EC
:10604000789410936B00109368001BBB90E080E085
:106050000E94722A182F81E090E00E94722A912FEC
:106060008F30984009F0B5C082E090E00E94722A1B
:10607000182F83E090E00E94722A912F909347019D
:106080008093460184E090E00E94722A182F85E0F8
:1060900090E00E94722A912F9093450180934401D1
:1060A00086E090E00E94722A8093430187E090E0AE
:1060B0000E94722A80934C0188E090E00E94722A2C
:1060C00080934B0189E090E00E94722A80934A01FC
:1060D0008AE090E00E94722A8093C0028BE090E0F8
:1060E0000E94722A91E0811101C090E090934901D1
:1060F0008CE090E00E94722A91E0811101C090E052
:10610000909348018DE090E00E94722A8093BD0236
:106110008EE090E00E94722A282E809342018FE048
:1061200090E00E94722A80934E0180E190E00E94EC
:10613000722A91E0811101C090E090939802A2E050
:106140008A2EA1E09A2EB0E5AB2EB1E0BB2E11E174
:10615000E12EF12C312C231409F447C010E000E0AB
:10616000C701800F911F0E94722AF501E00FF11FF5
:1061700080830F5F1F4F0630110591F7670126E0FE
:10618000C20ED11C3EE0E30EF11C3401C6010E9498
:10619000722A082F10E0102F0027F30111830083CB
:1061A0002601F2E04F0E511CC60101960E94722A90
:1061B000082BF301019311933F0162014E145F0418
:1061C00029F73394F8E08F0E911C26E0A20EB11C43
:1061D000C2CF68E090E080E00E946D286FE081E02F
:1061E00090E00E946D280E9481281091980280EC16
:1061F000111101C088EC0E94441E80EA111101C0F7
:1062000081EA0E94441E0E94DE1F909393028093B5
:1062100092020E9486209093B9028093B802009166
:106220004601109147011093B2020093B1028EE033
:106230000E945820BC0190E080E00E94E338609307
:1062400094027093950280939602909397020E9415
:106250001A200E94FA2320E030E040EA51E46091E5
:10626000B3027091B4028091B5029091B6020E947F
:10627000AB3A6B017C01B80190E080E00E94E3380A
:106280009B01AC01C701B6010E94DE3887FF04C044
:1062900090E080E00E94501D10929C0710929D0794
:1062A00010929E0710929F07412C512CEFE76E2E03
:1062B000E3E47E2E4092A0075092A1076092A207CD
:1062C0007092A307A0908807B09089078091A407D7
:1062D000F501C080D180E280F380882309F4C1C633
:1062E000A3019201C701B6010E94BF3B181634F505
:1062F000F501408251826282738280909007909073
:106300009107A0909207B0909307C090A007D090FB
:10631000A107E090A207F090A307A7019601C5018D
:10632000B4010E94BF3B1816C4F4C0929007D092EB
:106330009107E0929207F09293071FC020E030E0AF
:10634000A901C701B6010E94DE3887FFD6CFF5014B
:106350001082118212821382D0CFC0909C07D090FD
:106360009D07E0909E07F0909F07A7019601C50149
:10637000B4010E94DE3887FDD8CF81E08093A40766
:1063800083B181708093910289B190E0880F892F49
:10639000881F990B80939002209191029091900216
:1063A00081E0291380E080938F0284E690E090934F
:1063B0009F0280939E0280E293E090939D028093DF
:1063C0009C028AE090E090939B0280939A02000FD7
:1063D000111F1093AB020093AA020E94FF1D60934D
:1063E000AD027093AE028093AF029093B0020E9410
:1063F000C0200E94C0202090AA023090AB029101E0
:10640000359527953A8729873093B2022093B102B8
:1064100086E00E94BD1C482E81119EC08091A90279
:10642000882309F499C00E94C0200E94FF1D6B01BF
:106430007C01C092A502D092A602E092A702F0923F
:10644000A80286E00E94BD1C892B59F40E94FF1D02
:106450006C197D098E099F09643F71408105910582
:1064600080F30E94FF1D6C197D098E099F09643F0E
:1064700071408105910508F43FC48FEF90E00E94C0
:10648000501D0E94C020512C4AE0642E712C1092A5
:10649000A002852D0E94212C582EF7E0F81708F451
:1064A00038C0E82FF0E0E95AFD4C0C94D93B71322A
:1064B00019358F35F53503363D364B36553620E0E8
:1064C00030E0A901C701B6010E94DE3887FF55CF31
:1064D00010929007109291071092920710929307D2
:1064E0004CCF3EE1632E712C81E08093A002852D7C
:1064F0000E94212C582E22E0821709F434C228175A
:1065000008F4E8C0882309F410C131E0831709F4C6
:106510000FC10E94812881E08093B70229853A85C6
:106520003093B2022093B10284E690E090939F02F0
:1065300080939E0280E293E090939D0280939C0260
:106540008AE090E090939B0280939A02C1018E7F33
:106550009093AB028093AA024092A9028091BA0262
:10656000882309F110914A011123E9F00E94FF1DCF
:10657000C090A102D090A202E090A302F090A402E9
:106580006C197D098E099F0928EE33E040E050E048
:106590000E94793A211738F01092BA020E94C02066
:1065A00081E080934D018091B7028823E9F18091C9
:1065B000BB02882349F120E030E040EA51E46091D9
:1065C000B3027091B4028091B5029091B6020E941C
:1065D000AB3A6B017C016091B1027091B20290E024
:1065E00080E00E94E3389B01AC01C701B6010E9424
:1065F000DE3887FF04C090E080E00E94501D0E94BA
:10660000C02081E080934D011092B7021092BB022E
:106610001092BC020E94FF1D6093AD027093AE0207
:106620008093AF029093B0020E94FF1D0091AD02D3
:106630001091AE022091AF023091B002601B710B3D
:10664000820B930B20E63AEE40E050E00E94793A4C
:10665000122F2093AC028091BB0281110BC080915C
:106660004C01882339F0281728F081E08093BB0281
:106670000E94C0208091BC0281110BC080914B010F
:10668000882339F0181728F081E08093BC020E941B
:10669000C0200E9430290E94CD210E94FF1D8091C0
:1066A000B507362F381B832F9091B607992309F42D
:1066B00039C33093B7071092B60780E090E0892B7A
:1066C00009F499CE0E94F11B882309F494CE0E940C
:1066D000000091CE83E0581609F448C194E05912A5
:1066E00018CF80914201883008F0FECE91E0980FDB
:1066F000909342018093BD020E94DE20E091BD0292
:1067000028E0E29FF0011124EE5FFE4F88ED90E05B
:106710009183808324E331E03383228386E891E010
:106720009583848377826682DFCE0E945127DCCEF8
:106730008E010F5F1F4F812C912C5401839498EE92
:10674000E92E93E0F92ECC24C394D12CE091BD0224
:1067500024E0E29FF0011124C4010197E80FF91F22
:10676000EE0FFF1FEE5FFE4F808191819093B2028A
:106770008093B102E8ECF0E0F0939F02E0939E0278
:10678000F0929D02E0929C02D0929B02C0929A02EB
:10679000880F991F9093AB028093AA02F1E0F093C7
:1067A0004D0186E00E94BD1C21E0892B09F020E00C
:1067B000209399020E94731B22E02093BE070E943F
:1067C00030290E94CD211092B9071092B80710927B
:1067D000BB071092BA078EE291E30E94BB1FC5016E
:1067E000B4010E94F6248FE692E00E94A5248091D5
:1067F0004F011092B9071092B807882309F48BC093
:1068000080E190E09093BB078093BA0781E291E327
:106810000E94BB1F1092B9071092B807E0E2F0E0A7
:10682000F093BB07E093BA078AE191E30E94BB1F94
:106830006091AA027091AB0275956795072E000CC6
:10684000880B990B0E94F6240E94AE200E94271EFE
:1068500086E00E94BD1C892B09F0ACCF8091990283
:106860008111A8CF8091AA029091AB02959587954E
:10687000F801819391938F010E94C0206AE070E03B
:1068800080E090E00E94CD1DFFEF8F1A9F0AAF0AB3
:10689000BF0A24E082169104A104B10409F056CF86
:1068A0008FEF90E00E94501D8BEA94E00197F1F782
:1068B0000E941A200E94903B4B0178876F83C98009
:1068C000DA800B811C81C6014E968017910708F073
:1068D0000BCEED80FE80C8014E968E159F0508F008
:1068E00003CE87E08093A00280E00E94212C8823C1
:1068F00009F4FACDE091BD0238E0E39FF0011124E4
:10690000EE5FFE4FD182C08213830283F582E48260
:1069100097828682E9CD20E130E03093BB07209357
:10692000BA0784E191E30E94BB1F609194027091C9
:10693000950280919602909197020E94903B90E080
:1069400080E04AE00E94B2241092B9071092B80782
:1069500080E290E09093BB078093BA0788E091E3D0
:106960000E94BB1F71CF0E94DE20BECD87E08093C6
:10697000A00280914201813009F4B6CD80E00E94EE
:10698000212C882309F4B0CD1091BD020091420161
:10699000802F8150990BBC011817190639F411503A
:1069A0001093BD020150009342019ECD812F90E0D3
:1069B00086179707BCF7E6E01E9FD001112450E030
:1069C00040E09C012F5F3F4FFA01EA0FFB1FE05BA5
:1069D000FE4FF680F0824F5F5F4F46305105A1F7C2
:1069E00043E0220F331F4A95E1F7F901EE5FFE4FB6
:1069F0002081318153E0880F991F5A95E1F7DC011E
:106A0000AE5FBE4F11963C932E9382819381139675
:106A10009C938E9312978481958115969C938E9367
:106A200014978681978117969C938E9316971F5F74
:106A3000BDCF82E08093A00210E008E2C02ED12CEE
:106A400084E6A82EB12C90E2892E93E0992E24E1C1
:106A5000E22EF12C812F0E94212C182F813021F160
:106A600030F0823009F43FC00E94812810CD80911F
:106A7000460190914701B0929F02A0929E0290928F
:106A80009D0280929C0270929B0260929A02880FF3
:106A9000991F9093AB028093AA020E94F12B9093CE
:106AA000470180934601D6CF8091440190914501E2
:106AB000D0929F02C0929E02E0E9F1E0F0939D0225
:106AC000E0939C0270929B0260929A02880F991F39
:106AD0009093AB028093AA020E94F12B9093450100
:106AE00080934401B7CF8091430190E0F0929F02E0
:106AF000E0929E0228EC30E030939D0220939C02AD
:106B000070929B0260929A02880F991F9093AB0239
:106B10008093AA020E94F12B809343019BCF83E0D4
:106B20008093A00210E0812F0E94212C182F813029
:106B3000F1F1F8F0823009F097CF80914A0190E0AE
:106B400010929F0210929E02E8E6F1E0F0939D02FF
:106B5000E0939C0270929B0260929A02880F991FA8
:106B60009093AB028093AA020E94F12B80934A017A
:106B7000DACF80914C0190E010929F0210929E0219
:106B8000ECE3F0E0F0939D02E0939C0221E030E022
:106B900030939B0220939A02880F991F9093AB0227
:106BA0008093AA020E94F12B80934C01BCCF80916C
:106BB0004B0190E010929F0210929E02E8E7F0E0F5
:106BC000F0939D02E0939C0225E030E030939B021D
:106BD00020939A02880F991F9093AB028093AA0288
:106BE0000E94F12B80934B019ECF84E08093A00202
:106BF000809149010E94212C91E0811101C090E017
:106C00009093490144CC10E03AE0E32E45E0D42EC5
:106C100059E0C52EE092A002812F0E94212C182F4E
:106C2000882321F08130E1F000E009C0D092A00279
:106C30008091C0020E94212C8093C00201E0F0905C
:106C4000980280ECF11001C088EC0E94441E80EA9A
:106C5000F11001C081EA0E94441E0111DBCF04CF74
:106C6000C092A002809198020E94212C91E0811193
:106C700001C090E090939802E1CF86E08093A0025B
:106C8000809148010E94212C91E0811101C090E087
:106C900090934801FCCB88E08093A00280914E0144
:106CA0000E94212C80934E01F2CB86E00E94BD1CF5
:106CB00021E0892B09F020E0209399020E94731BA8
:106CC000EE24E39400E320E345E351E368E070E061
:106CD00088E290E00E94F11A0E94271E0E94AE20D6
:106CE00086E00E94BD1C892BC9F780919902811111
:106CF000F5CF0E94C020CBCB8091BA0291E08927CA
:106D00008093BA02882351F00E94FF1D6093A10274
:106D10007093A2028093A3029093A40281E08093D7
:106D2000B7021ACC9091B407391748F48F5F8917CE
:106D300008F0C3CC81E083BF889513BEBECC11E0C0
:106D40001093B6076093B5078091B0079091B10793
:106D500001969093B1078093B0078091C002882379
:106D600009F466C10E94731B01E020E440E870E072
:106D700060E090E080E00E94CF1A1093BE0710936D
:106D8000BD071092BC07E12C00E120E14CEC52E37E
:106D900070E060E090E080E00E94F11A83E190E012
:106DA0009093B9078093B80784E090E09093BB0775
:106DB0008093BA078091BD02E6E08E9FC001112446
:106DC000805B9E4F0E94A5248091BE029091BF02DD
:106DD000853F914008F0F7C08091BC028111F5C059
:106DE0008091BB028111F3C08091BA028111F1C080
:106DF00080914F018111EFC020E030E044E353E483
:106E000060916207709163078091640790916507B4
:106E10000E94DE3887FFE1C085E025E330E0309353
:106E2000B9072093B80721E030E03093BB072093E7
:106E3000BA0792E09093BE07C82ED12C90914E01D4
:106E4000CC0CDD1C9111CBC0F601E95CFD4F4081FB
:106E50005181E12C0EE02CE161E070E080E590E0F2
:106E60000E94F11AF601E75DFD4F40815181E12C4E
:106E700000E120E170E060E080E790E00E94F11A1C
:106E800081E08093BE0720E146E852E360E170E0D4
:106E900090E080E00E94F11A20E146E652E360E2D1
:106EA00070E090E080E00E94F11A03E110E010939E
:106EB000B9070093B80720E130E03093BB07209377
:106EC000BA070E941A2041E00E94202588EF0E9404
:106ED000D61F84E692E30E94BB1F1093B90700936C
:106EE000B80788E190E09093BB078093BA070E94AF
:106EF000DE1FBC0190E080E00E94E33820E030E03B
:106F00004AE754E40E94173B42E00E94202582E6B3
:106F100092E30E94BB1F1093B9070093B80780E269
:106F200090E09093BB078093BA076091B80270918C
:106F3000B90290E080E00E94E33820E030E04AE7C8
:106F400054E40E94173B41E00E94202580E692E332
:106F50000E94BB1F1093B9070093B80788E290E026
:106F60009093BB078093BA0789E592E30E94BB1F09
:106F700089E390E09093B9078093B80782E190E0AD
:106F80009093BB078093BA0784E08093BE0760911B
:106F9000BE027091BF02653F91E0790708F442C0DC
:106FA00085E592E30E94BB1F00E020E248E460E137
:106FB00070E087E390E00E94881E80E00E94F82540
:106FC0000E94271E7ACB80E028CF81E026CF82E086
:106FD00024CF83E022CF84E020CF86E01ECF833011
:106FE000C1F038F4813069F0823081F086EA92E3B2
:106FF0000AC08530A1F080F08630C1F78CEA92E3B8
:1070000002C088EC92E30E94BB1F2CCF82EC92E37B
:10701000FACF8CEB92E3F7CF86EB92E3F4CF81EBE0
:1070200092E3F1CF90E080E04AE00E94B224BCCF2E
:107030000E94731B8091BE029091BF02853FE1E0E8
:107040009E0710F087EE93E00E94742A00E023E090
:1070500040E860E370E090E080E00E94CF1A81E0B9
:10706000ADCFC0929007D0929107E0929207F09234
:107070009307E0918607F091870780819181A28133
:10708000B3818093940790939507A0939607B0934C
:10709000970720E030E04FE753E4C701B6010E94B4
:1070A000BF3B18160CF00BCA409290075092910704
:1070B000609292077092930760C98091A6079091A1
:1070C000A707009711F00C947B3C08951F93FC01D7
:1070D00099278827BC01E89411911032E9F31930FF
:1070E00010F01E30C8F31B3251F01D3249F4689481
:1070F00006C00E949F38610F711D811D911D119165
:1071000010531A30B0F33EF49095809570956195C8
:107110007F4F8F4F9F4F1F910895FB01DC0105901A
:107120000D920020E1F70895BB274A3031F49923EE
:1071300022F4BDE2909581959F4F0C94B538592F5C
:10714000482F372F262F660F771F881F991F660F2E
:10715000771F881F991F620F731F841F951F660F6B
:10716000771F881F991F0895BB27FB015527AA2762
:10717000880F991FAA1FA41710F0A41B83955051C4
:10718000B9F7A05DAA3308F0A95DA193009779F73C
:10719000B111B1931192CB010C94CE38DC01FC01FA
:1071A000672F71917723E1F7329704C07C916D933B
:1071B00070836291AE17BF07C8F308950E9420390B
:1071C00008F481E00895E89409C097FB3EF4909597
:1071D0008095709561957F4F8F4F9F4F9923A9F0B0
:1071E000F92F96E9BB279395F6958795779567953F
:1071F000B795F111F8CFFAF4BB0F11F460FF1BC083
:107200006F5F7F4F8F4F9F4F16C0882311F096E915
:1072100011C0772321F09EE8872F762F05C06623C3
:1072200071F096E8862F70E060E02AF09A95660F7C
:10723000771F881FDAF7880F9695879597F9089535
:10724000990F0008550FAA0BE0E8FEEF1616170677
:10725000E807F907C0F012161306E407F50798F0DF
:10726000621B730B840B950B39F40A2661F0232BF8
:10727000242B252B21F408950A2609F4A140A69574
:107280008FEF811D811D08950E9457390C94C839D4
:107290000E94BA3938F00E94C13920F0952311F0CC
:1072A0000C94B1390C94B73911240C94FC390E9418
:1072B000D93970F3959FC1F3950F50E0551F629F28
:1072C000F001729FBB27F00DB11D639FAA27F00D3F
:1072D000B11DAA1F649F6627B00DA11D661F829F66
:1072E0002227B00DA11D621F739FB00DA11D621F4B
:1072F000839FA00D611D221F749F3327A00D611D68
:10730000231F849F600D211D822F762F6A2F112449
:107310009F5750409AF0F1F088234AF0EE0FFF1F7C
:10732000BB1F661F771F881F91505040A9F79E3FD3
:10733000510580F00C94B1390C94FC395F3FE4F3B3
:10734000983ED4F3869577956795B795F795E79529
:107350009F5FC1F7FE2B880F911D9695879597F932
:10736000089597F99F6780E870E060E008959FEFC7
:1073700080EC089500240A941616170618060906CC
:10738000089500240A94121613061406050608959B
:10739000092E0394000C11F4882352F0BB0F40F423
:1073A000BF2B11F460FF04C06F5F7F4F8F4F9F4F63
:1073B000089557FD9058440F551F59F05F3F71F0E5
:1073C0004795880F97FB991F61F09F3F79F087954C
:1073D0000895121613061406551FF2CF4695F1DFD5
:1073E00008C0161617061806991FF1CF8695710565
:1073F000610508940895E894BB2766277727CB0199
:1074000097F90895F999FECF92BD81BDF89A992711
:1074100080B50895262FF999FECF1FBA92BD81BD80
:1074200020BD0FB6F894FA9AF99A0FBE0196089506
:10743000052E97FB1EF400940E942F3A57FD07D0AB
:107440000E94793A07FC03D04EF40C942F3A5095E1
:107450004095309521953F4F4F4F5F4F0895909540
:107460008095709561957F4F8F4F9F4F08950E9433
:107470009B3AA59F900DB49F900DA49F800D911DE8
:10748000112408952F923F924F925F926F927F92B4
:107490008F929F92AF92BF92CF92DF92EF92FF9224
:1074A0000F931F93CF93DF93CDB7DEB7CA1BDB0BD0
:1074B0000FB6F894DEBF0FBECDBF09942A88398875
:1074C00048885F846E847D848C849B84AA84B9847C
:1074D000C884DF80EE80FD800C811B81AA81B98188
:1074E000CE0FD11D0FB6F894DEBF0FBECDBFED019C
:1074F0000895A1E21A2EAA1BBB1BFD010DC0AA1FF5
:10750000BB1FEE1FFF1FA217B307E407F50720F00C
:10751000A21BB30BE40BF50B661F771F881F991F87
:107520001A9469F760957095809590959B01AC01D0
:10753000BD01CF010895A29FB001B39FC001A39FD9
:10754000700D811D1124911DB29F700D811D11249C
:10755000911D08955058BB27AA270E94C23A0C9447
:10756000C8390E94BA3938F00E94C13920F039F484
:107570009F3F19F426F40C94B7390EF4E095E7FB1D
:107580000C94B139E92F0E94D93958F3BA17620720
:1075900073078407950720F079F4A6F50C94FB395E
:1075A0000EF4E0950B2EBA2FA02D0B01B90190011E
:1075B0000C01CA01A0011124FF27591B99F0593F62
:1075C00050F4503E68F11A16F040A22F232F342FAA
:1075D0004427585FF3CF469537952795A795F040F8
:1075E0005395C9F77EF41F16BA0B620B730B840B0D
:1075F000BAF09150A1F0FF0FBB1F661F771F881FC5
:10760000C2F70EC0BA0F621F731F841F48F487951C
:1076100077956795B795F7959E3F08F0B0CF93950E
:10762000880F08F09927EE0F9795879508950E9487
:107630002B3B0C94C8390E94C13958F00E94BA39CA
:1076400040F029F45F3F29F00C94B13951110C94AA
:10765000FC390C94B7390E94D93968F39923B1F3F6
:10766000552391F3951B550BBB27AA276217730768
:10767000840738F09F5F5F4F220F331F441FAA1FFC
:10768000A9F335D00E2E3AF0E0E832D091505040B8
:10769000E695001CCAF72BD0FE2F29D0660F771F66
:1076A000881FBB1F261737074807AB07B0E809F04C
:1076B000BB0B802DBF01FF2793585F4F3AF09E3FD1
:1076C000510578F00C94B1390C94FC395F3FE4F328
:1076D000983ED4F3869577956795B795F7959F5F14
:1076E000C9F7880F911D9695879597F90895E1E060
:1076F000660F771F881FBB1F621773078407BA07BF
:1077000020F0621B730B840BBA0BEE1F88F7E09519
:1077100008950E94903B6894B1110C94FC3908952F
:107720000E94E13988F09F5798F0B92F9927B751F7
:10773000B0F0E1F0660F771F881F991F1AF0BA9515
:10774000C9F714C0B13091F00E94FB39B1E008953F
:107750000C94FB39672F782F8827B85F39F0B93F31
:10776000CCF3869577956795B395D9F73EF49095C8
:107770008095709561957F4F8F4F9F4F08950E9420
:10778000203908F48FEF08950E942039880B990B57
:107790000895DB018F939F930E94373ABF91AF9179
:1077A000A29F800D911DA39F900DB29F900D11245B
:1077B0000895EE0FFF1F0590F491E02D09940F93AB
:1077C0001F93CF93DF938230910510F482E090E015
:1077D000E091C207F091C30730E020E0B0E0A0E004
:1077E000309799F42115310509F44AC0281B390B4B
:1077F00024303105D8F58A819B816115710589F1A5
:10780000FB0193838283FE0111C04081518102817B
:10781000138148175907E0F04817590799F4109752
:1078200061F012960C93129713961C933296CF0127
:10783000DF91CF911F910F9108950093C20710938C
:10784000C307F4CF2115310551F04217530738F023
:10785000A901DB019A01BD01DF01F801C1CFEF01F0
:10786000F9CF9093C3078093C207CDCFFE01E20FFB
:10787000F31F819391932250310939832883D7CF05
:107880002091C0073091C107232B41F42091820140
:10789000309183013093C1072093C007209180016C
:1078A000309181012115310541F42DB73EB740914A
:1078B000840150918501241B350BE091C007F091A4
:1078C000C107E217F307A0F42E1B3F0B2817390757
:1078D00078F0AC014E5F5F4F2417350748F04E0F2C
:1078E0005F1F5093C1074093C007819391939FCF2F
:1078F000F0E0E0E09CCFCF93DF930097E9F0FC014C
:10790000329713821282A091C207B091C307ED0192
:1079100030E020E01097A1F420813181820F931F85
:107920002091C0073091C1072817390709F061C0BD
:10793000F093C107E093C007DF91CF910895EA016A
:10794000CE17DF07E8F54A815B819E01411551059D
:10795000B1F7E901FB83EA8349915991C40FD51F1F
:10796000EC17FD0761F4808191810296840F951FC9
:10797000E90199838883828193819B838A83F0E0E4
:10798000E0E012968D919C9113970097B9F52D9197
:107990003C911197CD010296820F931F2091C00751
:1079A0003091C1072817390739F6309751F51092F1
:1079B000C3071092C207B093C107A093C007BCCF02
:1079C000D383C28340815181840F951FC817D90783
:1079D00061F44E5F5F4F88819981480F591F518331
:1079E00040838A819B81938382832115310509F02D
:1079F000B0CFF093C307E093C2079ECFFD01DC0137
:107A0000C0CF13821282D7CFB0E0A0E0EAE0FDE35E
:107A10000C94443A8C01009751F4CB010E94DF3B57
:107A20008C01C801CDB7DEB7E0E10C94603AFC01EF
:107A3000E60FF71F9C0122503109E217F30708F403
:107A40009DC0D901CD91DC911197C617D70798F049
:107A5000C530D10530F3CE0104978617970708F398
:107A6000C61BD70B2297C193D1936D937C93CF0103
:107A70000E947B3CD6CF5B01AC1ABD0A4C018C0E38
:107A80009D1EA091C207B091C307512C412CF12C2F
:107A9000E12C109731F58091C0079091C1078815AE
:107AA000990509F05CC04616570608F058C0809149
:107AB000800190918101009741F48DB79EB740916C
:107AC000840150918501841B950BE817F90708F094
:107AD00055C0F093C107E093C007F901718360833B
:107AE000A0CF8D919C91119712966C90129713963E
:107AF0007C901397A815B90559F56C0142E0C40EA6
:107B0000D11CCA14DB0420F1AC014A195B09DA016B
:107B10001296159780F06282738251834083D90157
:107B20006D937C93E114F10471F0D7011396FC93EB
:107B3000EE93129776CF22968C0F9D1FF9019183B9
:107B40008083F301EFCFF093C307E093C20769CFBF
:107B50004816590608F42C017D01D3019ACFCB01B8
:107B60000E94DF3B7C01009749F0AE01B8010E9402
:107B7000C63DC8010E947B3C870153CF10E000E066
:107B800050CF81E090E0F8940C94D63DFB01DC01ED
:107B900002C001900D9241505040D8F70895FB016A
:107BA000DC0101900D920020E1F7089519E1C5E88C
:107BB000D9E104C0FE010E94D93B2196C638D10705
:107BC000C9F7F894FFCF01FFD800340186011E00E9
:107BD00000000000000000000000000000000000A5
:107BE0000000000000000000000000000000000095
:107BF0000000000000000000000000000000000085
:107C00000000000000000000013C9600400101015E
:107C1000280F050101014243312E3500000000000C
:107C20000000000000000000000000000000000054
:107C30000000000000000000000000000000000044
:107C40000000000000000000C40780004A0AFA0992
:107C5000AA095A090A09BA086A081A08CA074A0A80
:107C60007A072A07DA068A063A06EA059A054A05D5
:107C70003A069A05FA044A053A06AA045A040A047E
:107C8000BA036A031A03CA027A022A02DA01CA0292
:107C90007A028A013A013A06DA27BA269A257A2424
:107CA0005A233A221A21FA1FDA1EBA1D9A1CDA2721
:107CB0007A1B5A1A3A19DA271A18FA163A191A18A0
:107CC000DA15FA163A19BA149A137A125A113A10A6
:107CD0003A221A0FFA0DDA0CBA0B1A0FFA0D7A12B1
:107CE0009A0A3A1909060404020202020202039ADD
:107CF000297A295A2966323A291A29FA280A2BD2CE
:107D00002A9A2A622A2A2AF229BA29000000002780
:107D10001C871BB41B741CE51BC31BD71B00000076
:107D200000B91E871BDB1F861B6E616E00696E66C5
:087D3000006F7666002F33009E
:107E0000112484B714BE81FFF0D085E080938100F7
:107E100082E08093C00088E18093C10086E0809377
:107E2000C20080E18093C4008EE0C9D0259A86E02C
:107E300020E33CEF91E0309385002093840096BBD3
:107E4000B09BFECF1D9AA8958150A9F7CC24DD24C4
:107E500088248394B5E0AB2EA1E19A2EF3E0BF2EE7
:107E6000A2D0813461F49FD0082FAFD0023811F036
:107E7000013811F484E001C083E08DD089C08234E0
:107E800011F484E103C0853419F485E0A6D080C0E4
:107E9000853579F488D0E82EFF2485D0082F10E0AE
:107EA000102F00270E291F29000F111F8ED06801E7
:107EB0006FC0863521F484E090D080E0DECF843638
:107EC00009F040C070D06FD0082F6DD080E0C81688
:107ED00080E7D80618F4F601B7BEE895C0E0D1E017
:107EE00062D089930C17E1F7F0E0CF16F0E7DF06D8
:107EF00018F0F601B7BEE89568D007B600FCFDCFD4
:107F0000A601A0E0B1E02C9130E011968C91119780
:107F100090E0982F8827822B932B1296FA010C0160
:107F200087BEE89511244E5F5F4FF1E0A038BF0790
:107F300051F7F601A7BEE89507B600FCFDCF97BE46
:107F4000E89526C08437B1F42ED02DD0F82E2BD052
:107F50003CD0F601EF2C8F010F5F1F4F84911BD097
:107F6000EA94F801C1F70894C11CD11CFA94CF0C13
:107F7000D11C0EC0853739F428D08EE10CD085E9AC
:107F80000AD08FE07ACF813511F488E018D01DD067
:107F900080E101D065CF982F8091C00085FFFCCF94
:107FA0009093C60008958091C00087FFFCCF809118
:107FB000C00084FD01C0A8958091C6000895E0E648
:107FC000F0E098E1908380830895EDDF803219F02E
:107FD00088E0F5DFFFCF84E1DECF1F93182FE3DFCA
:107FE0001150E9F7F2DF1F91089580E0E8DFEE27F6
:047FF000FF270994CA
:027FFE00040479
:00000001FF
